:1000000002744E02778300000000000270B300000B
:100010000000000277E10000000000320000000054
:10002000000000023DF900000000000271E900003C
:1000300000000000000000000000000000000000C0
:100040005052343032207665722E3132382E332EB3
:1000500031204864773A482030362D30372D3035FE
:100060002030303A3038202075F00612011E22125E
:100070006DC975F00612011E126DCE2212006F12AC
:10008000006812006F12006812006F120068120000
:100090006F12006812006F75F01812011E22126DA7
:1000A000C975F04B12011E126DCE22755104123724
:1000B000BD1237D3126DC975F0C812011E126DCE74
:1000C000227551051237BD1237D312009E75F01EEE
:1000D00012011E12009E227551071237BD1237D32E
:1000E000120088227551061237BD1237D312008EC6
:1000F0002212007C12007C221200E41200E41200A2
:10010000E422C2A1C25812006F75F01212011ED271
:10011000A1C2582212006F75F01212011E22128223
:1001200047201607C0F0123207D0F0D5F0F0227049
:1001300004A243B322C0E01412013ED0E022C0E08A
:10014000030303540F28F8D0E0C0E0540704F5F08F
:10015000E213D5F0FCD0E0227003D3802830E7030F
:10016000C3802223F9C3137004A243801814C0E093
:10017000030303540F247AF8D0E0540704F5F0E2A7
:1001800013D5F0FCE992E022C0E024B5F8E21201B8
:10019000584004D0E0C322D0E024CBF58274003470
:1001A00000F583E01201A82220E702C322C2E7C0C3
:1001B000E0C2E0700AA243B3D0E030E001B322B461
:1001C0007E03C380F3B40204A22380ECB40404A22F
:1001D0002480E5B40604A22580DEB40804A22B80A6
:1001E000D7B40A04A20A80D0B40C0AE5764577C3D6
:1001F0006001D380C3B40E0512703580BBB4100704
:10020000A25E725DB380B1B41206A25D822680A8A0
:10021000B41406A25DB026809FB41604A25E809836
:10022000B418077400127DB6808EB41A07740112D8
:100230007DB68084B41C087402127DB60201B8B485
:100240001E087403127DB60201B8B42008740412AB
:100250007DB60201B8B422087405127DB60201B859
:10026000B424087406127DB60201B8B426087407D7
:10027000127DB60201B8D0E0C3221243A5E56D603D
:1002800013B401051232DD8008B402051232F38086
:1002900000756D00123207E5785440600B20A80805
:1002A000305505C25512332D127C0B22C2B612777F
:1002B0002C75380074031258B3E51E1258B3E51FAD
:1002C0001258B374571258B31202D5E5381258B306
:1002D0003099FDD3227885E6232354031258B3784E
:1002E00086E630E402240A540F1258B37885E6C437
:1002F000540375F00AA4F5F0E6540F25F01258B334
:100300007884E6C4540375F00AA4F5F0E6540F258A
:10031000F01258B37883E6C4540775F00AA4F5F0D8
:10032000E6540F25F01258B37882E6C4540775F0EE
:100330000AA4F5F0E6540F25F01258B37886E603C8
:10034000C454071258B32275F03212825FB2B5124C
:10035000825FB2B5D5F0F322D2A3C256D2A2C2595F
:10036000C2A1C258D2A4C257C2A0126DC91203477B
:10037000D2A0126DCE120347C2A0126DC91203475C
:10038000D2A0126DCE120347C2A0126DC91203474C
:10039000D2A0126DCE120347120347120347120375
:1003A0004712034722C0F075F0DCD5F005B2B51254
:1003B0006A1EC0F01205EFD0F030E7EED0F022AAAE
:1003C000F01203A5E5336530F5F0E534653145F00D
:1003D000600C1205168530338531341203A51205E1
:1003E000B41203A51205DC1203A51205238AF0221C
:1003F000AAF01203A5E5336530F5F0E53465314523
:10040000F0600C1205168530338531341203A512C5
:1004100005A01203A51205DC1203A51205238AF01C
:100420002279207530017531037532E09000E112B8
:1004300003A51205161203A5120574790075300183
:100440007531047532009001011203A512051612D0
:1004500003A512057479E075300175310575320018
:100460009002011203A51205161203A51205748548
:10047000303385313422AAF01203A5E5336530F517
:10048000F0E534653145F0600C1205168530338592
:1004900031341203A512055C8AF022AAF01203A5DA
:1004A000E5336530F5F0E534653145F0600C120553
:1004B000168530338531341203A51205448AF022A3
:1004C000C0F075F00833C297928300D297D5F0F54B
:1004D000D0F022C0F075F008C297D29700A2823304
:1004E000D5F0F5D0F022D2B7D297D283D282D2847F
:1004F00022E53133E5303322C3E5313322E53222C0
:100500001204C01204F11204C01204F81204C01242
:1005100004FD1204C0221204E6C2847453120500C2
:10052000D284221204E6C2847458120500D28422B6
:100530001204E6C2847454120500E41204C01204CA
:10054000D3D284221204E6C2847454120500E41249
:1005500004C01204D3F608D9F9D284221204E6C2E8
:10056000847454120500E41204C01204D3F208D9B2
:10057000F9D284221204E6C2847454120500E412F3
:1005800004C01204D3F0A3D9F9D284221204E6C025
:10059000E0C2847484120500D0E01204C0D2842228
:1005A0001204E6C2847484120500E61204C008D95D
:1005B000F9D284221204E6C2847484120500E21285
:1005C00004C008D9F9D284221204E6C284748412C9
:1005D0000500E01204C0A3D9F9D284221204E6C2B5
:1005E000847483120500D28412824712824722C289
:1005F0008474571204C01204D3D28422D283D282CC
:10060000D297D2B7D284B2B575F002128247D5F034
:10061000FAC2B7B2B575F002128247D5F0FAD2B776
:10062000B2B5227530017531DB7532001203A512A7
:1006300008BE7533FF7534FF22AE83AD8290DB00B8
:100640007F207404F97480F87530018583318582C8
:100650003212049B7880E66E702508E66D702008E3
:10066000E6601AB4FF028013167404F97480F875FA
:1006700030018583318582321203F0C322D322A355
:10068000A3A3A3DFBD80F490DB007F207404F97482
:1006900080F875300185833185823212049B788021
:1006A000E66E700908E66D700408E6FC22A3A3A3B9
:1006B000A3DF0A7CFF2290DB007F207BFF7404F91C
:1006C0007480F875300185833185823212049B78FD
:1006D00080E66E702C08E66D702708ECB4FF0D788C
:1006E0008076FF0876FF0876FF0874FFF67404F939
:1006F0007480F87530018583318582321203F0C32E
:1007000022BBFF107880E6B4FF0A08E6B4FF05C3F9
:1007100074209FFBA3A3A3A3DFA3BBFF02D322EB01
:10072000232354FC2400F5827583DB500205837873
:1007300080EEF608EDF608ECF608E4F67404F974B9
:1007400080F87530018583318582321203F0C3222F
:1007500075830075F08E753002858331753200C067
:10076000F0C0831203A51208BED0830583D0F0D554
:10077000F0E475830075F0DA7530038583317532E6
:1007800000C0F0C0831203A51208BED0830583D039
:10079000F0D5F0E47533FF7534FF22758300758260
:1007A0000075F08EC0F0C082C08375300285833141
:1007B0007532001203A5120516D083D082C082C004
:1007C000837530008582317532001203A51205DC75
:1007D000D083D08205830582D0F0D5F0C775830021
:1007E00075820075F0DAC0F0C082C0837530038571
:1007F00083317532001203A5120516D083D082C052
:1008000082C0837530018582317532001203A512D2
:1008100005DCD083D08205830582D0F0D5F0C77582
:1008200033FF7534FF2275830075820075F08EC02A
:10083000F0C082C0837530008583317532001203A9
:10084000A5120516D083D082C082C0837530028580
:1008500082317532001203A51205DCD083D08205E7
:10086000830582D0F0D5F0C775830075820075F0DE
:10087000DAC0F0C082C083753001858331753200E3
:100880001203A5120516D083D082C082C0837530B2
:10089000038582317532001203A51205DCD083D0A6
:1008A0008205830582D0F0D5F0C77533FF7534FF1C
:1008B000221204E6C2847450120500D2842212046B
:1008C000E6C2847481120500D284221204E6C28436
:1008D0007484120500E81204C0D9FAD28422F8798F
:1008E000001203A51208CBEAC0E08582308583316F
:1008F0007532001203A51205DCD0E0FA0583DAE7B1
:100900007533FF7534FF221204E6C2847454120555
:1009100000E41204C0E4C0E01204D3D0F025F0D902
:10092000F5D2842275830075820280067583007576
:100930008200E475F08D858230858331753200C088
:1009400082C083C0F0C0E01203A51205161203A5F1
:100950007900120907D0F025F0D0F0D083D08205BD
:1009600083D5F0D2858230858331753200C0E012A4
:1009700003A51205161203A57920120907D0F02548
:10098000F07533FF7534FF2275830075820380068E
:10099000758300758201E475F0DA858230858331D4
:1009A000753200C082C083C0F0C0E01203A51205FA
:1009B000161203A57900120907D0F025F0D0F0D067
:1009C00083D0820583D5F0D27533FF7534FF05E0FF
:1009D0002275830075F00075300085833175320013
:1009E000C0F0C0831203A51208BED0830583D0F0E7
:1009F000D5F0E47533FF7534FF75830075F0DA7553
:100A00003001858331753200C0F0C0831203A51216
:100A100008BED0830583D0F0D5F0E47533FF75347C
:100A2000FF2253590F53580F5318F053190FC2AFE9
:100A3000E5582324B1F8E5184519F608A61A055813
:100A400053580FE558B55905055953590FD2AFC33F
:100A5000E55895595002241024F450037563002280
:100A6000E559B558057400780022C33324B1F8E67F
:100A7000C0E008E6F8D0E02253580F53590FC2AF38
:100A8000E559B55804D2AFD322055953590FD2AF07
:100A9000C380F53008597885E6540FC0E0E6C454A9
:100AA0000375F00AA4D0F025F0FD7886E630E40264
:100AB000240A540FFE901A007F3C7404F97400F865
:100AC0007530018583318582321204767800E26DBB
:100AD000701708E26E701208E2C42354E0F5F07853
:100AE00086E6541F45F0F68006A3A3A3A3DFCB221E
:100AF00012772C120A9312773BFEAFF07DFF0DEDBB
:100B000030E70122D26575F004A424E1F582E5F016
:100B10003400F583C082C0837880E0F6A308E0F655
:100B2000A308E0F6A308E0F6D083D082788086831D
:100B30000886827880B6FF0708B6FF03020BB6C3AB
:100B4000E58233F582E58333F583E58224E0F5829F
:100B5000E5833405F5837882E6705B08E66057FB31
:100B60007402F97480F87530018583318582321200
:100B7000049BA3A37880E60856B4FF03020BB67863
:100B80008086F053F07F08E6C39EC5F09F401E703C
:100B900025E5F06018BD001E20431B7880E6A2E723
:100BA00020E713E5F024FA400DD27480097880E63E
:100BB000A2E79265DBAABD00028028ED14C0E00325
:100BC0000303540F247AF8D0E0540704FB7400D3D5
:100BD00033DBFD306505FBE24B8004F4FBE25BF2A6
:100BE000020AFEB265123254406E20316B20170BA0
:100BF000204205306562800320655D30653B204200
:100C00003878B4E2702D20731F78B2E2602B127432
:100C10000A6026F5F07518C0751909E5F0543F44CF
:100C200000F51A120A22800512740A600C78B2E2EA
:100C300078B4F2D274D273801FC274C273A2659268
:100C400042400D304312C24312330512524980080C
:100C5000204305D24312331B020AFE1204C01204C1
:100C6000F11204C01204F8D2E01204C01204FD1202
:100C700004C0221204E6C2847454120C5BE4120411
:100C8000C01204D3F608D9F9D284221204E6C28431
:100C90007484120C5BE61204C008D9F9D284229045
:100CA000FC00753004753100753200C082C0837558
:100CB0004BFA1203A512051685306C85316B790845
:100CC00078801203A5120C73120E9BD083D0827011
:100CD00044C082C08378848683088682120D4C408B
:100CE0002478828683088682120D4C4018120D6B80
:100CF000E582600AE569B56B0CE56AB56C07D083DF
:100D0000D082020D277882E6249AF6120EDE1203B4
:100D100058D083D0820531E53170020530A3E582D9
:100D200045837087120D2E7533FF7534FF2278824C
:100D30007600087600788476000876000876000849
:100D40007600756C04756B00120EBA22C082C083E7
:100D5000E5822400F582E5833480F5834005D08365
:100D6000D08222D083D08290000022E58275F008E4
:100D7000A4F582E5F0C58375F008A42583F583E525
:100D8000F03404F56AE5822400F582E5833400F549
:100D9000835002056A85836922120358D083D0826A
:100DA00022C082C083120E7470EF78828683088618
:100DB00082120D4C40E3120D6B12115578807600B3
:100DC0007884E518F608E519F608760008760074C8
:100DD00008F97480F8856A30858331858232120380
:100DE000F07404F97484F8856A3085833185823221
:100DF00012049B75F00478807984E667600280991C
:100E00000809D5F0F5120E7B78828683088682A3C6
:100E1000120D4C7882A68308A68278848683088681
:100E200082120D4C7882E66583700A08E66582704E
:100E300004A3120D4C7884A68308A682C06CC06BF4
:100E4000856A6C85696B120EBAD0E0D0F0B56B097B
:100E5000C5F0B56C028018C5F0C06CC06B85F06C35
:100E6000F56B7882E62499F6120EDED06BD06CD04A
:100E700083D08222120E7B120E9B22856C30856BF2
:100E8000317532001203A512051679087880120315
:100E9000A5120C73853033853134227885E6182607
:100EA0001826182618245566700F7885E6186618D7
:100EB00066186618661864996622120EC1120EDE54
:100EC000227885E6182618261826182455F67885DF
:100ED000E61866186618661866186499F622856C16
:100EE00030856B317532001203A51205161203A569
:100EF00079087880120C8B1203A51205DC1203A569
:100F000012052385303385313422120E7470307807
:100F100082E6C0E008E6C0E0088683088682C3D087
:100F2000E09582F582D0E09583F58350104582608C
:100F30000CE5822400F582E5833480F583C322909A
:100F40000000D322C2B6120F0AE433C0E0753800A5
:100F500074031258B3E51E1258B3E51F1258B37448
:100F6000531258B3D0E01258B374001258B374003F
:100F70001258B3E5831258B3E5821258B3E538121C
:100F800058B33099FD22C2B6E5366004F4FF800400
:100F9000FF120D2E75380074031258B3E51E125857
:100FA000B3E51F1258B374561258B3EF1258B3E595
:100FB000381258B33099FD227401C0E0788075F082
:100FC00008E4F608D5F0FBD0E0D322120F0A40E87F
:100FD00060E878848683088682120FDEC322C0828E
:100FE000C083E58275F008A4F582E5F0C58375F04D
:100FF00008A42583F583E5F03404F56AE58224002E
:10100000F582E5833400F5835002056A7408F974AB
:1010100080F8856A3085833185823212049BD083C3
:10102000D08222120F0A7F085005120D2E7F007801
:1010300082865A08865B08865C08865DC2B675386B
:101040000074031258B3E51E1258B3E51F1258B3CB
:1010500074541258B3E5361258B3EF1258B3E5364C
:10106000603CE55D655BF5F0E55C655A45F0600B5D
:10107000855D82855C83120FDE8003120FBA855D69
:1010800082855C83A3120D4C85825D85835C7880AC
:1010900075F008E61258B308D5F0F8D536C4E5382F
:1010A0001258B33099FDC322E5367007C2AF120F54
:1010B0000A5005E536F4800C7884A65C08A65D121B
:1010C0000EBAE536D2AFC0E0C2B67538007403126E
:1010D00058B3E51E1258B3E51F1258B37455125891
:1010E000B3D0E01258B3E5381258B33099FDD3228B
:1010F000C2B675380074031258B3E51E1258B3E532
:101100001F1258B374581258B37420232354FC048C
:101110001258B374201258B390DB007F207404F986
:101120007480F875300185833185823212049B7892
:1011300080E61258B308E61258B308E61258B3080E
:10114000E61258B308A3A3A3A3DFD2E5381258B31D
:101150003099FDD32212772C7886E630E402240AF7
:10116000540FC4F97885E6C4540375F00AA4F5F069
:10117000E6540F25F0C313497881F67885E692E7A7
:1011800054C0F97883E6C4540775F00AA4F5F0E674
:10119000540F25F049F97884E6C4540375F00AA485
:1011A000F5F0E6540F25F0F5F07882E6547023450B
:1011B000F07883F67882E9F622223044FD126DC978
:1011C00075F00612011E126DCE75F01412011EE5A7
:1011D00040C24422E42278807910E6B5F007080581
:1011E000F0D9F7E422740122C0E078807910F60883
:1011F00005E0D9FA7410F97480F87530037531DBA5
:101200007532001203F07410F97480F875300375AC
:1012100031DC7532001203F07410F97480F8753007
:10122000037531DB75320012049BD0F0C0F012114F
:10123000D6701E7410F97480F87530037531DC7542
:10124000320012049BD0F0C0F01211D67003D0F01F
:1012500022D0F022E51DC0E01211E8D0F07006E5C2
:10126000F0F41211E822785574FFF21213C8C20884
:101270001209906001221204217401F97455F87565
:1012800030017531037532A01204767410F9748A36
:10129000F87530017531037532C01204767410F997
:1012A000749AF87530017531037532D01204767472
:1012B00002F97467F87530017531CE753200120489
:1012C000767416F974B5F87530017531CE7532C083
:1012D00012047678B59000CB75F016E2F008A3D52D
:1012E000F0F97416F974B5F875300175310375327B
:1012F000A11204767408F97400F87530017531D2C2
:1013000075320012047678009002F475F008E2F06D
:1013100008A3D5F0F9D208E422798077E909E4A29C
:101320002692E0A22792E1A22892E2A22C92E3A2C6
:101330004292E4F709A73909A73A09A73B7404F9CF
:101340007480F875300275318E7532001203F02208
:10135000D242D243C221C227A227B392A5C222C23F
:1013600028A228B392A6C22AC22CA22CB392802211
:101370007404F97480F875300275318E753200127C
:10138000049B7880B6E9C908E6A2E092269220B3D1
:1013900092A7A2E192279221B392A5A2E29228926B
:1013A00022B392A6A2E3922A922CB39280A2E49254
:1013B00042788076FF7401F97480F87530027531D7
:1013C0008E7532001203F02278B575F016E4F2083B
:1013D000D5F0FB74FF78BDF278BEF222E8C0E07869
:1013E00062E2F571D0E0F822E8C0E07863E2F571DE
:1013F000D0E0F822E8C0E07864E2F571D0E0F822AD
:1014000075F00384B40104741A8017B402047422C2
:101410008010B40304742A8009B404047442800266
:10142000741A227403F9745FF875300075318C7585
:1014300032E5120476785FE21214007862F2786086
:10144000E21214007863F27861E21214007864F218
:10145000785FE224FD9201E224E292027401F974C1
:101460005EF875300075318C7532E2120476785E64
:10147000E224FD9204E224E29205227403F9745FEF
:10148000F875300075318C7532E51203BF7401F9BF
:10149000745EF875300075318C7532E21203BF222C
:1014A0007980774809774E0977800977A07404F925
:1014B0007480F875300075318D7532201203F07428
:1014C00004F97480F875300275318D75322012037D
:1014D000F0227404F97480F875300075318D75321E
:1014E0002012049B7982E7648022E4A21C92E0A28D
:1014F0001D92E1A21E92E2A22992E37980F7740183
:10150000F97480F875300075318C7532E81203F08B
:10151000227401F97480F875300075318C7532E8E9
:1015200012049B7980E7A2E0921CA2E1921DA2E244
:10153000921EA2E39229227980E4A22D92E0A22EAB
:1015400092E1A22F92E2A21492E392E492E5A231F8
:1015500092E692E7F709E4A23092E0A23292E1A289
:101560003392E2A23492E3A23692E6A23792E7F7F0
:1015700009E4A23892E0A23A92E2A23B92E3A23CB2
:1015800092E4A23D92E5A23E92E7F709E578F7746E
:1015900004F97480F875300075318C7532EC1203E3
:1015A000F07980E579F4F709E57AF4F709E57BF459
:1015B000F77403F97480F875300075318C7532E971
:1015C0001203F0227404F97480F875300075318CC0
:1015D0007532EC12049B7980E7A2E0922DA2E19291
:1015E0002EA2E2922FA2E39214A2E69231A2E70980
:1015F000E7A2E09230A2E19232A2E29233A2E39219
:1016000034A2E69236A2E7923709E7A2E09238A226
:10161000E2923AA2E3923BA2E4923CA2E5923DA27E
:10162000E6A2E7923E09E7F5787403F97480F8754D
:10163000300075318C7532E912049B7980E7F4F53E
:101640007909E7F4F57A09E7F4F57B227980F774F4
:1016500001F97480F875300075318C7532E412032D
:10166000F0227401F97480F875300075318C753290
:10167000E412049B7980E7227401F9744FF8753005
:101680000075318C7532FC1203BF227401F9744F5E
:10169000F875300075318C7532FC12047622784F63
:1016A000E270067850F208F22275F000303C0475C2
:1016B000F03CA4AAF075F008A4FBACF0EA75F008C1
:1016C000A42CFAC374FD9BFB74FF9A7850F2EB08CC
:1016D000F2227401F97452F875300075318D75324B
:1016E000001203BF227401F97452F875300075318D
:1016F0008D753200120476227402F97470F8753018
:101700000075318C7532FD1204767402F97472F82A
:1017100075300075318D753201120476227402F92C
:101720007470F875300075318C7532FD1203BF741A
:1017300002F97472F875300075318D75320112033B
:10174000BF227401F97456F875300075318C75320A
:10175000F01203BF7401F97457F875300075318CBD
:101760007532F41203BF7401F97458F875300075BE
:10177000318C7532F61203BF7401F97459F8753063
:101780000075318C7532F21203BF227401F9745660
:10179000F875300075318C7532F01204767401F9E9
:1017A0007457F875300075318C7532F41204767404
:1017B00001F97458F875300075318C7532F61204E1
:1017C000767401F97459F875300075318C7532F200
:1017D000120476227401F97439F875300075318C71
:1017E0007532F81203F07401F9743AF87530007527
:1017F000318C7532FA1203F07401F9743BF87530CC
:101800000075318C7532FB1203F0227401F97439C2
:10181000F875300075318C7532F812049B7401F93B
:10182000743AF875300075318C7532FA12049B7475
:1018300001F9743BF875300075318C7532FB120478
:101840009B227402F9741EF875300075318C753264
:10185000E01203F0227402F9741EF875300075313D
:101860008C7532E012049B22E57B54026003757094
:101870000378A17984AA7080021819E7F5F06654FC
:101880000F700E18E7C4F5F066540F7004DAEAE43E
:1018900022E6540FC5F0540FC395F092077401224D
:1018A0007885791F7A03E6C4540FF309E6540FF3E1
:1018B0000908DAF2791F78A47A06E6540FF6E3668F
:1018C00070080908DAF4E4C24922792478A97A0672
:1018D000C3E3961918DAFA9207792478A97A06E30D
:1018E000540FB40F08E6540FB40F108008E6540FDD
:1018F000B40F0B80061819DAE680CB740122C3E31B
:1019000096B40902801214600FC3E3F5F0E695F077
:10191000B4090280031470E3E9B41F04E4D249223D
:101920001918E366540F60F080D11218A0701D30B2
:10193000491A20301875185085831985821A120AA1
:10194000227549B4757C00D245D248E42204227441
:1019500008F97480F875300075318C7532C0120446
:101960009B0218687408F97480F875300075318C22
:101970007532C012049B12192A227405F97480F87A
:1019800075300075318C7532C01203F0227403F982
:101990007485F875300075318C7532C51203F022EC
:1019A000C082C083E5822420F582E583347DF583FF
:1019B0007401F9743CF875300085833185823212E8
:1019C000049BD083D082C082C083E58275F008A4D6
:1019D0002420F582500205F0A8F0E58375F008A4F4
:1019E000282400F5837408F97480F8753000858325
:1019F0003185823212049BD083D082124D1522C0D1
:101A000082C083E58275F008A42420F58250020587
:101A1000F0A8F0E58375F008A4282400F583740885
:101A2000F97498F875300085833185823212049BF1
:101A3000D083D08222C082C083E58275F008A424BE
:101A400020F582500205F0A8F0E58375F008A4287F
:101A50002400F5837406F97480F8753000858331AD
:101A600085823212049BD083D082227405F974805F
:101A7000F875300075310075322012049B02186829
:101A80009000001219A0121868223008F3751B008C
:101A9000751C0075679F75680FE567251BC2E0F52B
:101AA00082E568351CF583C082C083E5822400F599
:101AB00082E583341BF5837402F97480F875300174
:101AC00085833185823212049B78808683088682E2
:101AD0001219A01218687005D0F0D0F022D083D06F
:101AE00082C3E58313F583E58213F582200714E5AD
:101AF0008245836022E58224FFF567E58334FFF5A4
:101B0000688007A385821B85831CC3E567951BE559
:101B100068951C400280827401223008397410F9E3
:101B20007480F87530017531CE75322012049B78BF
:101B300098798075F00AE7B4FF02801AB43C120865
:101B400009D5F0F2900FE878C3E2F53C7854F2E45E
:101B50002266540F60E97401229000001219A0124D
:101B6000192A2278A4E6540FB40F03021BFD2008A3
:101B70000280E6751B00751C0075679F75680FE590
:101B800067251BC2E0F582E568351CF583C082C07D
:101B900083E5822400F582E583343BF5837402F902
:101BA0007480F875300185833185823212049B7808
:101BB0008086830886821219A012192A7005D0F037
:101BC000D0F022D083D082C3E58313F583E582135E
:101BD000F582200714E58245836022E58224FFF523
:101BE00067E58334FFF5688007A385821B85831C26
:101BF000C3E567951BE568951C400280827401224D
:101C000078987A0579ACE6540FC4F5F008E6540FDD
:101C100045F0F70809DAEF2275F01E128247D5F079
:101C2000FA1200E475F00F128247D5F0FA1200E4C0
:101C300075F00F128247D5F0FA1200E422120094D8
:101C4000B2B575F00F128247D5F0FA30B7EF22D255
:101C500016D2A3C256C2A2D259D2A1C258D2A4C28D
:101C600057121C3D121C18121EFC12662A1276C84E
:101C7000120D2E120623C2A3C256C2A2C259C2A17D
:101C8000C258D2A4C257126DF14005C2AF0273C24E
:101C9000120094B2B575F00F128247D5F0FA80E6C3
:101CA000C2A3C256C2A2C259C2A1C258D2B775F0CD
:101CB00002128247D5F0FA20B744126DF15002802B
:101CC0008ED216D2A3C256C2A2D259D2A1C258D223
:101CD000A4C257121C3DD216126670401CC2A3C289
:101CE00056C2A2C259C2A1C258D2A4C257121E27BC
:101CF00012662A120D2E120623C2AF0273C2126D93
:101D0000CEC01D12092CD0F0703AC3E51D95F0F538
:101D10007D121DC51214D26019D21690000012193E
:101D2000A0121E2712662A120D2E120623B2B51219
:101D30001DC5121266E57B540870081276A5500383
:101D4000121D8322D2A3C256D2A2C259C2A1C25826
:101D5000D2A4C257C216754BFAC2A075F0C812823F
:101D600047D5F0FA126DC9D2A075F0C8128247D5D6
:101D7000F0FA126DCED2B712825F20B7C7021CBA3A
:101D8000020000D2B712825F30B7F5D2A3C256D29A
:101D9000A2C259C2A1C258D2A4C257C216754BFAE8
:101DA000C2A075F014128247D5F0FA126DC9D2A004
:101DB00075F014128247D5F0FA126DCE12687312C4
:101DC00076A540BF221215111215C4121662A2E0A8
:101DD000923FA2E19240A2E2924112168B1216E5C6
:101DE00012178B12180B1216F87401F974B2F875E9
:101DF00030017531CE75323012047678B2E2B4FF1C
:101E000002E4F27401F974B3F87530017531CE75DE
:101E1000323112047678B3E2B4FF02E4F2121855BC
:101E200012142312169E22D216C2A3C256C2A2C2F6
:101E300059C2A1C258D2A4C257C01EC01F788090F8
:101E400000007A08E6F008A3DAFA121EFC1276C83F
:101E500078809000007A08E0F608A3DAFA90000093
:101E600012659912197A12198DD01FD01E121842BC
:101E700022751E30751F30D21CC21DC21EC229C25F
:101E80002DC22EC22FC214C231C230D232C233C2CE
:101E900034C236C237C238C23AC23BC23CC23DC26B
:101EA0003E757800757900757A00757B08787074D6
:101EB00022F2087400F278727406F2087400F2C21A
:101EC0003FC240C241784F7404F278527409F278EC
:101ED000567401F278577402F278587404F2785903
:101EE0007404F2753907753A00753B007401785E29
:101EF000F2785FF2E408F208F2C208221209D11265
:101F00001E711218421214EA121537C2E0A23F9253
:101F1000E0A24092E1A24192E212164C121678120F
:101F200016D21217421217D412171D12147B121454
:101F3000A0126E4B22305B04C25B800975F00C204E
:101F4000B205D5F0FAD322C322E8C0E0E9C0E0EA46
:101F5000C0E0200437200134121F35502575510090
:101F6000785FE2600C75F003128247D5F0FA123404
:101F7000E2785EE2600C75F003128247D5F0FA1247
:101F80003643D0E0FAD0E0F9D0E0F8222002222057
:101F9000051F3069EDC082C083E56F700812784F6D
:101FA0004003121FC81213DC12781FD083D0828026
:101FB000D13069CEC082C083E56F700312201E123B
:101FC0007928D083D08280BA30030C300409D264DF
:101FD000C263785E021FE03001F4D263C264785FAE
:101FE000E2B40F028013B41007124EB7D251802D05
:101FF00075F00384E5F0B40007124F9AD251801DAA
:10200000B40107124E32D2508013B40210124DA9FF
:10201000400B784DE583F208E582F2D2522230037C
:102020000C300509D264C263785E0220363002F4B7
:10203000D263C264785FE275F00384E5F0B400090E
:1020400012514D4020D251801CB4010912517540EB
:1020500014D2508010125178400B784DE583F2086D
:10206000E582F2D25222D2538008C2531220D87590
:102070003D00C215D25B754BFA7440301602740CE9
:10208000F548C251C244E5486039121F4920513316
:1020900075F003128247D5F0FA12027A2016032057
:1020A00015183044E120531B7548601211BAB40B67
:1020B0000D75F008128247D5F0FAD2518005122032
:1020C000CB80C3C250D2AF754BFA22533D07F8E51F
:1020D0003D24A4C8F6053D2278A475F00874FFF6E7
:1020E00008D5F0FB22305009201B03D21B22C2501E
:1020F00022C21B22D2538004D25BC253C215754B3D
:10210000FAD21A7440301602740CF5481220D875B1
:102110003D00C251C250C244C252C25412027A207F
:10212000160320152D121F49205129205026205218
:102130002330442D785EE27004C24480242053147E
:102140007548601211BAB40B1275F008128247D5A7
:10215000F0FAD251757C03754BFA22757C0312207C
:10216000CBE54860F23054FD80B0C0E01222EDD0E3
:10217000E04021302E0320431B205E18C0E0126D8A
:10218000D3126DC1D0E0203A091281F075181012F7
:102190000A22D322203A091281F0751820120A224D
:1021A000C322D20B7518C0751900751A01120A22C4
:1021B000302619205D1C20380DC2AF754CFF754DBF
:1021C000F8D2AF126DB77852E2F5472220360312EB
:1021D000227022E51A543F44C0F51A751908C25EF0
:1021E000C25D205C46126DADD25B803FE51A543F64
:1021F0004480F51A751908D25E80E5E51A543F440B
:1022000040F51A751908D25DC25E205C1E126DADD4
:10221000D25B8017E51A543F4400F51A751908D2AD
:102220005DC25E8000205C03126DC17518C0120A89
:10223000222230150122C0E074108004C0E0741125
:1022400078A4760A0875F00A84F608A6F0753D03AE
:10225000D0E078AEF2087405F2D21522C20B7547B1
:1022600000C2477518C0751900751A02120A222299
:10227000757C00D2457549B475185075190F751ADB
:10228000FF120A222275186075190F751AFF120ABB
:1022900022757F03C245C2482275187075190F75E3
:1022A0001AFF120A22757F0322126E4BE51A543F61
:1022B0004400F51A75190B7518C0120A2222787499
:1022C000F208F21238877518C0751900751A501285
:1022D0000A2222400C305C08C25C205D03126DAD06
:1022E00022205CFC126DD3126DC1D25C2212262416
:1022F000400D1229DF4008122D9A40031231582256
:1023000012262F400D1229EA4008122DA540031273
:10231000316322A290301C01B3785AE233F22210CA
:1023200076030226CD301608C3785AE4F202263D21
:10233000E57A541060033043EF785AE260EF0460AE
:10234000030226CB201F0320234DD223300819C0BF
:10235000E0C082C0837400120188D083D082D0E0B4
:1023600040030226CB0223687856E224B0401CC00A
:1023700082C083902582E225E00493F5F0E225E017
:1023800093D083D082C0F0C0E0E222E2751890754D
:102390001909F51A120A220226CB126B2B1200D74A
:1023A0000226CB74011221A20226CB740112216AEB
:1023B00040E80226CBC2431222850226CBD270759A
:1023C0006E0502238CC0E07401127D6DD0E0022303
:1023D0008C20430320370CC0E07404127D6DD0E0E4
:1023E00002238C0226CB743D0224AF02238CC0E072
:1023F000E57B54047005D0E002238CD0E00226CBAC
:10240000C0E0D374011222D3D0E002238C02238CCB
:1024100002238C74001222320226CB741012223254
:102420000226CB74111222320226CB7420122232E1
:102430000226CB7401F97480F875300075318C7503
:1024400032F112049B7880E61222320226CB74010C
:10245000F97480F875300075318C7532F112049B77
:102460007880E612223C0226CB30741C78B3E260FE
:102470001778B4F27518C07519097401543F448077
:10248000F51A120A2202239A0226CB3074FAE47853
:10249000B4F27518C07519097401543F4440F51A17
:1024A000120A2202239A751A011222A902239A20E3
:1024B0004308D24312229902239AC2431222850270
:1024C000239AE57854106007E41222BE02239A0290
:1024D00026CBE5785410600874FF1222BE02239ABE
:1024E0000226CB751A011221D30226CB751A0112CE
:1024F00022140226CB751A011221FB0226CB751A73
:10250000011221EC0226CB7400127D6D740112823F
:102510009302239A7400127D9974011282A20223FD
:102520009A7400127DB640EC0225077402127D6D8C
:1025300074011282B102239A7402127D99740112FD
:1025400082C002239A7402127DB640EC02252B74DD
:1025500003127D6D74011282CF02239A7403127DDF
:102560009974011282DE02239A7403127DB640EC44
:1025700002254F3043030224BA0226CB2043FA023D
:1025800024B226CB23A323AB23B5238C238C238C0B
:1025900023BD23C523D123E6238C23EB23EE240084
:1025A000238C238C238C238C238C238C238C238CB3
:1025B000238C238C238C238C238C238C238C238CA3
:1025C000238C238C238C238C238C238C238C238C93
:1025D000238C238C238C238C238C238C238C238C83
:1025E000238C238C238C240D24102413241B2423BC
:1025F000242B2433244E2469248B24A624AF24C204
:1026000024D224E324EC24F524FE250725142521D7
:10261000252B25382545254F255C2569238C2573D9
:10262000257C238C7856E2B40B03A22322C32220FC
:1026300043097856E2B40D03A22322C322201F06C9
:102640002023030226CBC223300819C0E0C082C079
:10265000837400120188D083D082D0E04003022628
:10266000CB0226647856E260DAB4010612225C02DC
:1026700026CBB402030226CBB40307D2431222991D
:102680008049B40908204336303733803EB40A020B
:10269000743DB40D0BE57B54047030740D0226BEFE
:1026A000B40E0BC374011222D3740E0226BEC0E016
:1026B00024CED0E05008C0E024B0D0E0500D751812
:1026C000A0751909F51A120A228000D27622A29169
:1026D000301D01B3785BE233F222107603022A88C0
:1026E000301608C3785BE4F20229F8E57A542060DA
:1026F000033043EF785BE260EF046003022A862038
:102700001F0320244DD224300819C0E0C082C083AA
:102710007401120188D083D082D0E04003022A865F
:102720000227237857E224B0401CC082C08390293E
:102730003DE225E00493F5F0E225E093D083D082DA
:10274000C0F0C0E0E222E275189075190AF51A127D
:102750000A22022A86126B2B1200D7022A867402E2
:102760001221A2022A86740212216A40E8022A86F5
:10277000C243122285022A86D270756E050227474F
:10278000C0E07401127D6DD0E00227472043032092
:10279000370CC0E07404127D6DD0E0022747022A96
:1027A00086743D02286A022747C0E0E57B54047026
:1027B00005D0E0022747D0E0022A86C0E0D37402A9
:1027C0001222D3D0E002274702274702274774008E
:1027D000122232022A867410122232022A867411C0
:1027E000122232022A867420122232022A867401B0
:1027F000F97480F875300075318C7532F512049BD0
:102800007880E6122232022A867401F97480F87503
:10281000300075318C7532F512049B7880E61222F7
:102820003C022A8630741C78B3E2601778B4F275E3
:1028300018C07519097402543F4480F51A120A220F
:10284000022755022A863074FAE478B4F27518C06B
:102850007519097402543F4440F51A120A220227DE
:1028600055751A021222A9022755204308D2431295
:102870002299022755C243122285022755E5785432
:10288000106007E41222BE022755022A86E578541A
:1028900010600874FF1222BE022755022A86751A9C
:1028A000021221D3022A86751A02122214022A86E3
:1028B000751A021221FB022A86751A021221EC02F5
:1028C0002A867400127D6D74021282930227557459
:1028D00000127D9974021282A20227557400127DA3
:1028E000B640EC0228C27402127D6D74021282B1ED
:1028F0000227557402127D9974021282C002275574
:102900007402127DB640EC0228E67403127D6D74E9
:10291000021282CF0227557403127D99740212822B
:10292000DE0227557403127DB640EC02290A3043BB
:1029300003022875022A862043FA02286D2A862778
:102940005E2766277027472747274727782780274E
:102950008C27A1274727A627A927BB274727472733
:1029600047274727472747274727472747274727F7
:1029700047274727472747274727472747274727E7
:1029800047274727472747274727472747274727D7
:1029900047274727472747274727472747274727C7
:1029A0004727C827CB27CE27D627DE27E627EE28BE
:1029B00009282428462861286A287D288D289E28F1
:1029C000A728B028B928C228CF28DC28E628F32970
:1029D00000290A291729242747292E29372747782C
:1029E00057E2B40B03A22422C3222043097857E202
:1029F000B40D03A22422C322201F06202403022A8E
:102A000086C224300819C0E0C082C083740112015C
:102A100088D083D082D0E04003022A86022A1F7821
:102A200057E260DAB4010612225C022A86B402037D
:102A3000022A86B40307D2431222998049B40908B6
:102A4000204336303733803EB40A02743DB40D0B58
:102A5000E57B54047030740D022A79B40E0BC374F4
:102A6000021222D3740E022A79C0E024CED0E050A4
:102A700008C0E024B0D0E0500D7518A075190AF513
:102A80001A120A228000D27622A292301E01B37856
:102A90005CE233F222107603022E43301608C3782C
:102AA0005CE4F2022DB3E57A544060033043EF78E2
:102AB0005CE260EF046003022E41201F0320254DDD
:102AC000D225300819C0E0C082C083740212018888
:102AD000D083D082D0E04003022E41022ADE785813
:102AE000E224B0401CC082C083902CF8E225E004B0
:102AF00093F5F0E225E093D083D082C0F0C0E0E20D
:102B000022E275189075190CF51A120A22022E414C
:102B1000126B2B1200D7022E4174031221A2022E37
:102B200041740312216A40E8022E41C243122285F9
:102B3000022E41D270756E05022B02C0E0740112A4
:102B40007D6DD0E0022B0220430320370CC0E074DF
:102B500004127D6DD0E0022B02022E41743D022C46
:102B600025022B02C0E0E57B54047005D0E0022B67
:102B700002D0E0022E41C0E0D374031222D3D0E091
:102B8000022B02022B02022B027400122232022EAE
:102B9000417410122232022E417411122232022E7E
:102BA000417420122232022E417401F97480F875AA
:102BB000300075318C7532F712049B7880E6122252
:102BC00032022E417401F97480F875300075318C31
:102BD0007532F712049B7880E612223C022E4130B7
:102BE000741C78B3E2601778B4F27518C0751909CF
:102BF0007403543F4480F51A120A22022B10022E4D
:102C0000413074FAE478B4F27518C0751909740388
:102C1000543F4440F51A120A22022B10751A03126F
:102C200022A9022B10204308D243122299022B1012
:102C3000C243122285022B10E57854106007E4127B
:102C400022BE022B10022E41E5785410600874FF5A
:102C50001222BE022B10022E41751A031221D3023A
:102C60002E41751A03122214022E41751A031221E5
:102C7000FB022E41751A031221EC022E4174001240
:102C80007D6D7403128293022B107400127D99746F
:102C9000031282A2022B107400127DB640EC022CAB
:102CA0007D7402127D6D74031282B1022B107402C6
:102CB000127D9974031282C0022B107402127DB629
:102CC00040EC022CA17403127D6D74031282CF02BA
:102CD0002B107403127D9974031282DE022B107480
:102CE00003127DB640EC022CC5304303022C3002A7
:102CF0002E412043FA022C282E412B192B212B2B5D
:102D00002B022B022B022B332B3B2B472B5C2B0252
:102D10002B612B642B762B022B022B022B022B0216
:102D20002B022B022B022B022B022B022B022B023B
:102D30002B022B022B022B022B022B022B022B022B
:102D40002B022B022B022B022B022B022B022B021B
:102D50002B022B022B022B022B022B022B832B8606
:102D60002B892B912B992BA12BA92BC42BDF2C0169
:102D70002C1C2C252C382C482C592C622C6B2C7498
:102D80002C7D2C8A2C972CA12CAE2CBB2CC52CD2A4
:102D90002CDF2B022CE92CF22B027858E2B40B0327
:102DA000A22522C3222043097858E2B40D03A225AC
:102DB00022C322201F06202503022E41C2253008EF
:102DC00019C0E0C082C0837402120188D083D0820F
:102DD000D0E04003022E41022DDA7858E260DAB4E6
:102DE000010612225C022E41B40203022E41B403FA
:102DF00007D2431222998049B4090820433630375C
:102E000033803EB40A02743DB40D0BE57B5404706C
:102E100030740D022E34B40E0BC374031222D3741B
:102E20000E022E34C0E024CED0E05008C0E024B022
:102E3000D0E0500D7518A075190CF51A120A2280F1
:102E400000D27622A285302901B3785DE233F222E6
:102E5000107603023206301608C3785DE4F20231C0
:102E600071E57A548060033043EF785DE260EF04EF
:102E70006003023204201F03202B4DD22B3008198F
:102E8000C0E0C082C083740A120188D083D082D08F
:102E9000E04003023204022E997859E224B0401C2B
:102EA000C082C0839030B6E225E00493F5F0E225BD
:102EB000E093D083D082C0F0C0E0E222E2751890A7
:102EC00075190DF51A120A22023204126B2B120028
:102ED000D702320474041221A202320474041221B3
:102EE0006A40E8023204C243122285023204D270E0
:102EF000756E05022EBDC0E07401127D6DD0E0023A
:102F00002EBD20430320370CC0E07404127D6DD029
:102F1000E0022EBD023204743D022FE302320402AD
:102F20002EBDC0E0E57B54047005D0E0022EBDD07C
:102F3000E0023204C0E0D374041222D3D0E0022EA7
:102F4000BD022EBD022EBD74001222320232047464
:102F5000101222320232047411122232023204742C
:102F6000201222320232047401F97480F8753000A4
:102F700075318C7532F312049B7880E6122232028E
:102F800032047401F97480F875300075318C753233
:102F9000F312049B7880E612223C02320430741C47
:102FA00078B3E2601778B4F27518C0751909740423
:102FB000543F4480F51A120A22022ECB023204300A
:102FC00074FAE478B4F27518C07519097404543FA2
:102FD0004440F51A120A22022ECB751A041222A9B5
:102FE000022ECB204308D243122299022ECBC24399
:102FF000122285022ECBE57854106007E41222BE1F
:10300000022ECB023204E5785410600874FF1222BD
:10301000BE022ECB023204751A041221D3023204EE
:10302000751A04122214023204751A041221FB02CA
:103030003204751A041221EC0232047400127D6D00
:103040007404128293022ECB7400127D99740412C0
:1030500082A2022ECB7400127DB640EC02303B748B
:1030600002127D6D74041282B1022ECB7402127DA5
:103070009974041282C0022ECB7402127DB640EC09
:1030800002305F7403127D6D74041282CF022ECB66
:103090007403127D9974041282DE022ECB74031223
:1030A0007DB640EC023083304303022FEE0232043F
:1030B0002043FA022FE632042ED42EDC2EE62EBD5B
:1030C0002EBD2EBD2EEE2EF62F022F172EBD2F1C3D
:1030D0002F222F342EBD2EBD2EBD2EBD2EBD2EBDBA
:1030E0002EBD2EBD2EBD2EBD2EBD2EBD2EBD2EBD88
:1030F0002EBD2EBD2EBD2EBD2EBD2EBD2EBD2EBD78
:103100002EBD2EBD2EBD2EBD2EBD2EBD2EBD2EBD67
:103110002EBD2EBD2EBD2EBD2EBD2F412F442F47BF
:103120002F4F2F572F5F2F672F822F9D2FBF2FDA03
:103130002FE32FF630063017302030293032303B65
:1031400030483055305F306C307930833090309D6E
:103150002EBD30A730B02EBD7859E2B40B03A22BA0
:1031600022C3222043097859E2B40D03A22B22C3C3
:1031700022201F06202B03023204C22B300819C064
:10318000E0C082C083740A120188D083D082D0E06C
:1031900040030232040231987859E260DAB4010641
:1031A00012225C023204B40203023204B40307D2D6
:1031B00043122299804EB4090820433B30373880AF
:1031C00043B40A02743DB40C028039B40D0BE57BA4
:1031D00054047030740D0231F7B40E0BC374041232
:1031E00022D3740E0231F7C0E024CED0E05008C0E4
:1031F000E024B0D0E0500D7518A075190DF51A1225
:103200000A228000D27622E5785440601AE579548B
:1032100002700612231312231FE57954047006125C
:1032200026CE1226DA800C12231312231F1226CE6A
:103230001226DA122A89122A95122E44122E50C210
:103240001F204A0122C24A7518C0751900751A5408
:10325000120A2222E8C0E07856E264036018785728
:10326000E2640360117858E26403600A7859E2640A
:10327000036003C38001D3D0E0F8221201143008A8
:103280000C1267D1400390FFF112681B22C052124A
:1032900032ABD052223008131267D1400390FFF1B5
:1032A00012681B5005F55212687222E552700575BE
:1032B00052108023B41005755211801BB41105758E
:1032C00052208013B420057552FF800BB4FF0575A2
:1032D000520080037552FF126923E55222C24375E2
:1032E000186075190F751AFA120A22757F03C24504
:1032F000C24822D24375187075190F751AFA120A4E
:1033000022757F0322C24375186075190F751AE084
:10331000120A22757F03C245C24822D24375187033
:1033200075190F751AE0120A22757F0322E4A2268E
:1033300092E0A22792E1A22892E2A22C92E3F573F6
:103340007574051237FD7403500412398322123943
:103350005D7891E6C0E0E57954026012D0E0C0E00B
:10336000540712338BD0E0C0E0540712338BE57959
:1033700054046014D0E0C0E0C454071233B0D0E06D
:10338000C0E0C454071233B0D0E022A223301C01A5
:10339000B34007D320E10A0233AFC320E203023374
:1033A000AF301C01B3E4500114785AF212231F22EB
:1033B000A224301D01B34007D320E10A0233D4C355
:1033C00020E2030233D4301D01B3E4500114785BD2
:1033D000F21226DA22B40207205107C250C252026A
:1033E0003463C082C08390EA60E53D606324FB40A3
:1033F0005F78A4E6540F758300F582D53D028050B6
:1034000075F00AA4F58275830008E6540F2582F54D
:1034100082D53D02803AE58275F00AA4F58285F0F6
:103420008308E62582F58250020583D53D0280207F
:10343000E58275F00AA4F582C0F0E58375F00AA470
:10344000D0F025F0F58308E62582F5825002058349
:10345000784DE583F208E582F2C251C250D252D0D3
:1034600083D08222C289C28BD293C2B422C0F075AB
:10347000F0FAD5F0FD75F064D5F0FDD0F0221234ED
:103480006D12346D12346D12346D12346D12346D50
:1034900022D293C2B475F00512825F20B206128266
:1034A0005F30B203D5F0F112825F22C0F075F008F0
:1034B000A2E7B392B4C29312346DC2B4D293123461
:1034C0006DC0E0E430B201040030B201040030B25B
:1034D0000104D36003D5E001C3D0E033D5F0D1D0EF
:1034E000F022D293C2B4D2B212346DC29312347E9F
:1034F000D29312347E20160330641C789076010833
:103500007480F608A2A3B392E4F6749008F608F665
:1035100008F608F602355778907603087680087426
:1035200080A25692E5A2A3B392E4201608A2599273
:10353000E1A22692E0F608748020161220640FE5BE
:103540005154074480A25892E5A2A1B392E4F60830
:103550007480F608F608F675F00778907E007F0014
:10356000E62EFEE61234ABF62FFF08D5F0F2EED3CE
:10357000331234ABF8EFD3336870647890B6FF5FE2
:103580000561E56124FE501475610220180ED21801
:103590007518C0751900751A03120A2220160878CA
:1035A0005FE2600330640302363F7896E620E35919
:1035B00020E24920E1277891E6B6002108B64209C9
:1035C00008E6D263123A8F8076B6551108B6000D20
:1035D00008794DE6F30809E6F3D252D2638060E53C
:1035E000616017D56114301811C2187518C07519AB
:1035F00000751A04120A22757E0380437891863D75
:1036000008D25179A47A04800B7891D25075700554
:1036100079987A05D26375F00FE6C4540FF755F028
:10362000F5F009E6540FF755F0F5F00908DAEAE588
:10363000F0B40F051977EEC250785FE21233D5125D
:10364000349122D293C2B4D2B212346DC2931234E6
:103650007ED29312347E20161F3063237890761129
:10366000087480F608A2A3B392E4F6749008F608F2
:10367000F608F608F60236C8789076150236837892
:10368000907613087680087480A25692E5A2A3B3C0
:1036900092E4206314A25792E1A2A4B392E0201610
:1036A00008A25992E1A22692E0F608748020630FE6
:1036B000E55154074480A25892E5A2A1B392E4F6E2
:1036C000087480F608F608F675F00778907E007F9B
:1036D00000E62EFEE61234ABF62FFF08D5F0F2EE30
:1036E000D3331234ABF8EFD3336870627890B6FFFF
:1036F0005D0560E56024FE501475600220190ED24D
:10370000197518C0751900751A05120A22785EE23B
:1037100060033063030237B97896E620E36520E260
:103720005520E1487891E6B6002208B6420A08E63C
:10373000D264123A8F0237B9B6551108B6000D0897
:10374000794DE6F30809E6F3D252D264806BE56066
:103750006017D56014301911C2197518C075190099
:10376000751A06120A22757E030237B9D26478915F
:103770008640D24480437891863D08D25179A47A1C
:1037800004800B7891D25075700579987A05D264CF
:1037900075F00FE6C4540FF755F0F5F009E6540F35
:1037A000F755F0F5F00908DAEAE5F0B40F051977F6
:1037B000EEC250785EE21233D512349122785FE285
:1037C000601024FD400C75F003128247D5F0FA1208
:1037D00034E222785EE2601024FD400C75F00312A2
:1037E0008247D5F0FA12364322C0E030630C7518D8
:1037F000B0751900751A00120A22D0E022D293C2C5
:10380000B4D2B212346DC29312347ED29312347E8B
:103810007890E574540FC44407F608E57323A2E3D7
:1038200092E5A2E292E3542AD2E7F608E573A2E316
:1038300092E1A2E492E3542AD2E7F608E573A2E605
:1038400092E1A2E792E3540AD2E7F6748008F60800
:10385000F608F675F00778907E007F00E62EFEE60B
:103860001234ABF62FFF08D5F0F2EED3331234AB9F
:10387000F8EFD33368700B7890B6FF06123491C31B
:103880008004123491D3227574087874E2F57312AF
:1038900037FD7400400512395D8003123983757459
:1038A000097875E2F5731237FD7401400512395D30
:1038B00080031239832222E578542060F97574045C
:1038C0007573FF1237FD74025004123983221239C6
:1038D0005D78937948E6F30809E6F308794AE6F358
:1038E0000809E6F37891E6A2E092E25414F5F008B4
:1038F000E623A2E592E0540345F0F5F0784CE2654A
:10390000F0C0E0E5F0F2D0E030E21FC0E0C0F0E54A
:10391000F075F04930E20375F04A7518C07519006A
:1039200085F01A120A22D0F0D0E054037003023955
:103930005CE5F05403B4030575F0488013B4020548
:1039400075F047800BB4000575F04B800375F04CA3
:103950007518C075190085F01A120A2222F5F02494
:1039600042F8E2B40205227402F22250FA7402F222
:10397000E5F02432F5F07518C075190085F01A12BB
:103980000A2222F5F02442F8E2601AD5E016F2E5A8
:10399000F0243CF5F07518C075190085F01A120A6C
:1039A00022757E03F222D293C2B4D2B212346DC217
:1039B0009312347ED29312347E7890E574540FC4FF
:1039C0004403F6087680087480A25692E5A2A3B359
:1039D00092E4A25992E1A22692E0F6087480A258DD
:1039E00092E5A2A1B392E4F6087480F608F608F610
:1039F00075F00778907E007F00E62EFEE61234AB6D
:103A0000F62FFF08D5F0F2EED3331234ABF8EFD334
:103A1000336870717890B6FF6C7896E620E33020BA
:103A2000E22020E1607891E6B6005A08B655110808
:103A3000B6005208794DE6F30809E6F3D252804AFF
:103A400080437891863D08D25179A47A04800B781E
:103A500091D25075700579987A0575F00FE6C454C7
:103A60000FF755F0F5F009E6540FF755F0F5F009AA
:103A700008DAEAE5F0B40F051977EEC2507865E28E
:103A80001233D58005123491D322123491C322B45B
:103A9000FF15D270756E051237E97518C0751900DB
:103AA000751A07120A2222B4BC03023AC0B4BD033D
:103AB000023AF2B4BE03023B24B4BF03023B5622D7
:103AC0002063147408F97480F87530017531CE756F
:103AD000324012049B80127408F97480F87530012A
:103AE0007531CE75324812049B74117888F6123BFA
:103AF00088222063147408F97480F87530017531D8
:103B0000CE75325012049B80127408F97480F875D7
:103B100030017531CE75325812049B74127888F6D4
:103B2000123B88222063147408F97480F875300100
:103B30007531CE75326012049B80127408F974805E
:103B4000F87530017531CE75326812049B741378A4
:103B500088F6123B88222063147408F97480F87583
:103B600030017531CE75327012049B80127408F9E1
:103B70007480F87530017531CE75327812049B74FB
:103B8000147888F6123B88227881E61201584004A6
:103B9000741ED3227882E61201A8400C741FD3222F
:103BA000126B2B1200D7C3227880E660F9B4FF08AD
:103BB000D270756E05023DB0B40212203A0312377E
:103BC000E97888E612216A400280DB80D3B4090CD0
:103BD000C0E07404127D6DD0E0023DB0B4380878C6
:103BE00083E6123DC180BFB439087883E6123DCB2D
:103BF00080B4B43A253074201237E978B3E278B44F
:103C0000F2788886F07518C0751909E5F0543F44BC
:103C100080F51A120A228088808CB43B223074F816
:103C20001237E9E478B4F2788886F07518C075190F
:103C300009E5F0543F4440F51A120A22023BA0B4B1
:103C40003C0D1237E97888861A1222A9023BA0B4EB
:103C50003D311237E9204314D24375187075190F9E
:103C6000751AE9120A22757F03023BA0C243751838
:103C70006075190F751AE9120A22757F03125249ED
:103C8000023BA0B43E13E5785410600A1237E9E411
:103C9000123DD0023BA0023BA6B43F14E57854107D
:103CA000600B1237E974FF123DD0023BA0023BA625
:103CB000B4400D1237E97888861A1221D3023BA04E
:103CC000B4410D1237E97888861A122214023BA0FB
:103CD000B4420D1237E97888861A1221FB023BA004
:103CE000B4430D1237E97888861A1221EC023BA002
:103CF000B4440E7400127D6D7888E6128293023B04
:103D0000A0B4450E7400127D997888E61282A20252
:103D10003BA0B446097400127DB640E880D5B44794
:103D20000E7402127D6D7888E61282B1023BA0B457
:103D3000480E7402127D997888E61282C0023BA078
:103D4000B449097402127DB640E880D5B44A0E74B5
:103D500003127D6D7888E61282CF023BA0B44B0E31
:103D60007403127D997888E61282DE023BA0B44C7F
:103D7000097403127DB640E880D5B44D181282ED67
:103D80007888E6543F4480F51A75190B7518C012EF
:103D90000A22023BA0B44E0C3043061237E9023C23
:103DA0006C023BA0B44F092043F71237E9023C589C
:103DB0001237E97518C0751907F51A120A22023B65
:103DC000A61222327888E678AFF22212223C80F4E2
:103DD0007874F208F21238877888E6543F44C0F5C8
:103DE0001A75190B7518C0020A22700575631E80BA
:103DF00002D21122C298C299322016F830991EC2FE
:103E000099204F057535008014C0F0C0E0C0D07512
:103E1000D010E535124124D0D0D0E0D0F020980168
:103E200032C298204FFAC0F0C0E0C0D075D0103038
:103E30004E05C24E754100E54524FE40037545021E
:103E4000E54120E71FE54154072324E6C0E0740064
:103E5000343FC0E0E5992205412544F544D0D0D057
:103E6000E0D0F032543F232324E7C0E07400343E16
:103E7000C0E0E59922156280DE80DCD562FBB544A6
:103E800012D20FE8C0E078AA74FAF2D0E0F87541D7
:103E90000080CA023FF6B462FA80BC80BAB42AF34A
:103EA00080B5F56224C6E56240E924F5E56250E399
:103EB000056280A37818F21562809C7819F2156269
:103EC0008095781AF21562808E781BF215628087D1
:103ED000781CF215628080781DF21562023E5778D8
:103EE0001EF21562023E5702400E00023E9600028C
:103EF0003E9B00023E9D00023EA200023E75000273
:103F00003E7500023E7500023E7500023EB400029E
:103F10003EBB00023EC200023EC900023ED000028B
:103F20003ED700023EDF00023E7B00023E7B0002E5
:103F30003E7B00023E7B00023E7B00023E7B000295
:103F40003E7B00023E7B00023E7B00023E7B000285
:103F50003E7B00023E7B00023E7B00023E7B000275
:103F60003E7B00023E7B00023E7B00023E7B000265
:103F70003E7B00023E7B00023E7B00023E7B000255
:103F80003E7B00023E7B00023E7B00023E7B000245
:103F90003E7B00023E7B00023E7B00023E7B000235
:103FA0003E7B00023E7B00023E7B00023E7B000225
:103FB0003E7B00023E7B00023E7B00023E7B000215
:103FC0003E7B00023E7B00023E7B00023E7B000205
:103FD0003E7B00023E7B00023E7B00023E7B0002F5
:103FE0003E7B0002400E800E802D8031803580386F
:103FF000803B80488046B409097544007541000241
:104000003E57B44209754400754180023E577544DD
:1040100000754100023E5DB51EDC023E57B51FD65D
:10402000023E57F542023E57F543023E57B544C69D
:1040300075452012403E754100023E5D80D08542AC
:1040400037127219D24FE537B44603025933B447D9
:104050000412722F22B4500E8543361271F4C2AC92
:10406000C24F75720722B45312854336E543700A76
:104070001271F4C2ACC24F75720222B4540E854361
:10408000361271F4C2ACC24F75720122B4550E855E
:1040900043361271F4C2ACC24F75720322B4560E8D
:1040A0008543361271F4C2ACC24F75720422B45704
:1040B0000E8543361271F4C2ACC24F75720522B43C
:1040C000580E8543361271F4C2ACC24F7572062287
:1040D000B44E3D854336E543B4000B1271F4C2ACD7
:1040E000C24F75720822B4010B1271F4C2ACC24FF8
:1040F00075720922B4020B1271F4C2ACC24F757210
:104100000E22B4030B1271F4C2ACC24F75720F22AF
:1041100024BF24E6400485433622C24F22C53825F9
:1041200038C53822E53524F0400EE535232443C058
:10413000E074003441C0E022759906C24F75350025
:10414000D2B622802F8034803680388039803E80FD
:104150004680488051804F804D804B804680508003
:104160000E0241EB753503F59912411D053522E527
:1041700036024199753800740380ECE51E80E8E54D
:104180001F80E402424FE53875350F80DA120A606D
:10419000123DEA883680D0E53680C9E536A24392E2
:1041A000E080C1753503A8360536E676FF80B8E5B0
:1041B00036C313603214700BA22392E0B392E14431
:1041C0000480D614700BA22492E0B392E1440880DC
:1041D000C8147008A22592E0440C80BD147008A297
:1041E0002B92E0440C80B274FC80AEE5361470254E
:1041F0007408305C12305D044406809D305E0444D7
:1042000003809644078092A25D92E0A25E92E1A2B2
:104210002692E280841470157410A22392E0A224E6
:1042200092E1A22592E2A22B92E302419914700D31
:104230007418A21892E0A21992E102419914700B2D
:10424000A25F92E0A26192E2024199E4024199E503
:1042500037B44106753504024167B44212E5366051
:1042600003301103120A7875631E7442024164B46C
:10427000440280F8B44B028003024314E53654F83C
:10428000B4083EE5365407700B751A191221D3E5B0
:1042900037024349B4010B751A191221ECE53702B4
:1042A0004349B4020B751A191221FBE53702434941
:1042B000B4030B751A19122214E53702434902415F
:1042C00038B42003024138B42826E53620E008300F
:1042D000430B1252498006204303127445E536A26F
:1042E000E09243756D015003756D02E5370241643C
:1042F000B4300CE53654F8127D6DE537024164B4F4
:10430000380CE53654F8127D99E5370241640241D4
:1043100038024138B4430FB5360375460375350787
:104320007536AC024167B44A26E536701F205E1C24
:10433000205C087419126DD3126DC17518107519AF
:104340000F751AF0120A22E537024164024138B4AF
:104350004506753506024167B4510675350C0241B4
:1043600067B44D0EE53612807BE5375002B2E702A6
:10437000426CB44C0675350E024167B4460280C9E2
:10438000B4470280C4B44F08C245C246C24780B990
:10439000B4590FE536700B857D36745975350D02AD
:1043A0004167024138E572B4000122B40717C2AC7C
:1043B000128277128277D299127053C24FD2B612FC
:1043C00071F40244C9B40117C2AC12827712827729
:1043D000D299121023C24FD2B61271F40244C9B45A
:1043E0000317C2AC128277128277D2991210A8C238
:1043F0004FD2B61271F40244C9B40217C2AC128291
:1044000077128277D299120F44C24FD2B61271F44A
:104410000244C9B40417C2AC128277128277D299CF
:10442000120F86C24FD2B61271F40244C9B40517F6
:10443000C2AC128277128277D2991202ACC24FD2EA
:10444000B61271F40244C9B40617C2AC12827712D4
:104450008277D2991210F0C24FD2B61271F4024490
:10446000C9B40817C2AC128277128277D299126C43
:104470006BC24FD2B61271F40244C9B40917C2AC70
:10448000128277128277D299126BEFC24FD2B61294
:1044900071F40244C9B40E17C2AC1282771282774B
:1044A000D299126CF8C24FD2B61271F40244C9B458
:1044B0000F17C2AC128277128277D299126D3AC26C
:1044C0004FD2B61271F40244C975720022E564C27B
:1044D000676002D267E552F553C24820520C205063
:1044E0001B305103024602024AD8120102784DE203
:1044F000F58308E2F5821219A00246BF12010212EA
:104500001C00121A8A6017121B1A603C1237E975D8
:10451000182075190F751AEC120A2202454B2063F8
:1045200005205F0A8003206105124B84501AC08267
:10453000C0831200E412206AD083D08230510CE58F
:104540003D600812192A70030246BF754A3CD546E1
:10455000177518C0751900751A53120A227546038B
:10456000757C00D2467549B4024AC5D270756E0595
:104570001237E97518C0751900751A07120A2275E5
:1045800051041237BD1237D375F06412011E024A6E
:10459000D8206324E57A540860CE300818C0E0C003
:1045A00082C0837411120188D083D082D0E040028F
:1045B00080B90245D90245D9E579548060AA30080E
:1045C00018C0E0C082C0837410120188D083D082EA
:1045D000D0E0400280950245D91222ED401E205EB7
:1045E00015302E03204309900FE9124AE1024AD800
:1045F000124A5D024AD8124A63024AD8124A690234
:104600004AD8120102E53D608878A4E6B40A0302A4
:10461000523B121B63707D206305205F5080032096
:10462000614B124B844046206325300819C0E0C01E
:1046300082C0837413120188D083D082D0E04003FB
:104640000246BF0246490246BF124A3902454B3074
:104650000818C0E0C082C0837412120188D083D0D1
:1046600082D0E040030246BF80DF0246BF1200E472
:10467000C082C0831220F8D083D082305013C08211
:10468000C083120102121C00D083D082121868600D
:104690002E02454B785E206402785FE2B40F0A1266
:1046A0004E6FC251D2500244FFB4100280F1123753
:1046B000E975182075190F751AEB120A2280D2308D
:1046C0006330300819C0E0C082C083740C120188C6
:1046D000D083D082D0E040030246F20246DE7574F9
:1046E000027860E27865F21213E8124FE850030294
:1046F000454B306430300819C0E0C082C083740D6F
:10470000120188D083D082D0E040030247250247BF
:10471000117574037861E27865F21213F4124FE8B0
:10472000500302454B1273EF4003123464E53C041E
:10473000700302454B754A00754603C247C24620C6
:104740004802C245C082C083124C2BD083D0825015
:1047500006124A78024AD8C082C083120639D08332
:10476000D0825006124A78024AD8E58224CEE583E8
:1047700034FF5017124B724012C212C2131232543D
:104780005006124A69024AD802496E1222ED5012AE
:10479000124A69024912124A63024912124A5D0220
:1047A0004912205EF1302E032043F1306303785428
:1047B000E2306402E53C12015840030247C7024858
:1047C0000B124A570249123008F73014F4303DF109
:1047D00012513F4036A263303E01B3502E300818CC
:1047E000C0E0C082C0837409120188D083D082D017
:1047F000E0400280CC0247F8C082C083126FDFD055
:1048000083D0825006124A6E024912301425D239E2
:10481000300819C0E0C082C0837414120188D083AC
:10482000D082D0E0400302482E02482CC2391251F7
:104830003F50030248A3126F8BA2E09212A2E192B2
:1048400013A263303E01B3C0E09206501E127035D1
:10485000501930390EE4A21292E0A21392E1B40290
:10486000028008D0E0124A45024912D0E0B40005A7
:10487000200622802BB4012220061A7518C0751953
:1048800000751A09120A22203906124A73024912C7
:10489000124B35800E126EDE8009B402ED2006DB6D
:1048A000126F3630085812513F4053300819C0E09B
:1048B000C082C0837408120188D083D082D0E040C7
:1048C000030248FE0248C720671AA26392668583E6
:1048D00065858266124B31C263C2641200F875644A
:1048E00002024AD8756400E5836565F5F0E58265E6
:1048F0006645F07006124A7D0249121251DC124AD6
:10490000E1E5785410600BC082C083124D3BD08328
:10491000D082124B7B5009124D1530E103024AD868
:1049200012325440F8C2A1D258D2A4C257755100D5
:104930001237BD1237D31219A0C082C0831220F8DB
:10494000D083D08220520920501720511C024AD80F
:10495000120102784DE2B5830D08E2B582080249E2
:104960006E1218686008024AC512192A70F83014CD
:1049700024E4A21292E0A21392E1B40305126F6242
:104980008013B40205126EDE800BB40105126F367F
:104990008003126EB5300819C0E0C082C08374066F
:1049A000120188D083D082D0E04003024AC5024978
:1049B000B1E57854016022E5824583601C306303D1
:1049C0007854E2306402E53C12015840030249D3B6
:1049D0000249D9124A4B024AD8122300500F124AF8
:1049E0005175F01E12011E1200C1024AD8B24312C4
:1049F00037E930432075187085831985821A120AA9
:104A000022757F03C2A3C256D2A1C258D2A4C257F4
:104A1000127445801E75186085831985821A120AE2
:104A200022757F03D2A3C256D2A1C258C2A4C257D4
:104A30001252491200D7024AD8126B21024A801240
:104A40006B21024A80126B21024A80126B21024ABA
:104A500080126B21024A80126B21024A80126B2164
:104A6000024A80126B21024A80126B218012126B63
:104A700021800D126B218008126B218003126B21A3
:104A80007564007565FF7566FFD2771237E9751892
:104A90002085831985821A120A221200C1C2772248
:104AA000E5795408700320631BE55204601614F581
:104AB000F07855E265F0600C7518C07519018552E3
:104AC0001A120A2222126B21D2771200ABC277751A
:104AD00064007565FF7566FFC251C250E553F5521B
:104AE0002230430EC2A3C256C2A2C259D2A4C25798
:104AF000800CD2A3C256C2A2C259C2A4C257A2639A
:104B0000920AD209126B21741C126DD3126DC1E589
:104B1000785440600620A80312332D1237E9124A58
:104B2000A075181085831985821A120A221200D7DF
:104B300022126B2122126B2175F03212011E227497
:104B400008F97480F87530017531037532901204DC
:104B50009B7885E6085608560460141200E412207B
:104B60006A305109E53D600512192A6002C322D35B
:104B70002222E582249CE58334FF22E582249CE501
:104B80008334FF22A240E58245836010E582249CA5
:104B9000E58334FF5004A23F8002A24122E5822532
:104BA00082F582E5833583F583E5822582F582E50A
:104BB000833583F583E5822400F582E583345BF554
:104BC000837404F97400F87530018583318582326D
:104BD000120476227885E654C0F5837886E630E4C0
:104BE00002240A2323543C4583F5837885E6C45484
:104BF0000375F00AA4F5F0E6540F25F0030303F55E
:104C0000F053F0E085F08254034583F5837884E621
:104C1000C4540375F00AA4F5F0E6540F25F045825C
:104C2000F58222C39582E5F095832212513F50030D
:104C3000024CB3124B9D7800E2B4FF03024CB31256
:104C4000772C124BD47880A68308A6827800E2F5F0
:104C50008308E2F58208E2F5F008E2124C23502BBB
:104C60007800E2F58308E2F582788086F008E612A3
:104C70004C2350417802E2F58308E2F58278808681
:104C8000F008E6124C23402D024CB37800E2F58385
:104C900008E2F582788086F008E6124C2340167808
:104CA00002E2F58308E2F582788086F008E6124C8D
:104CB000235002C322D322C3E58233F582E5833336
:104CC000F583E5822400F582E583349AF583740246
:104CD000F97453F875300185833185823212047678
:104CE00022C3E58233F582E58333F583E582240030
:104CF000F582E583349AF5837402F97453F87530BC
:104D0000018583318582321203BF2278537400F209
:104D100008E4F2801E3008F3C082C083124CB7D082
:104D200083D082E5822418E58334FC40067853E280
:104D30004402F27854E2F5F018E222E5822400F50C
:104D400082E58334BAF5837401F97480F875300113
:104D500085833185823212049B7880E6604223236A
:104D6000C0E05403F5F0D0E054FC2400F582E5F0F7
:104D700034CAF5837404F97480F875300185833181
:104D800085823212049B7880E60886F07874F208F7
:104D9000E5F0F275F002128247D5F0FA1238872258
:104DA00074FF7874F208F280EAE571B4220575F0B8
:104DB000048013B42A0575F006800BB4420575F023
:104DC0000C800375F002782EE2540F704F08D5F076
:104DD000F7E2540F75F00AA4F58275830008E254D7
:104DE0000F2582F582E58275F00AA4F58285F083AD
:104DF00008E22582F58250020583E58275F00AA457
:104E0000F582C0F0E58375F00AA4D0F025F0F583B3
:104E100008E22582F58250020583C322D322782E30
:104E2000E2600BF5F008E2240A4005D5F0F7C32252
:104E3000D322782EE571B4220A757004799A75F040
:104E4000088024B42A0A757005799875F00A8017CD
:104E5000B4420C757005799875F00A78348008753D
:104E60007003799C75F006E2F70809D5F0F922C0C5
:104E700082C08378989002E175F00AE0F608A3D525
:104E8000F0F99002EBE0F570D083D08222C082C0AE
:104E90008378989002E175F00AE6F008A3D5F0F95E
:104EA000E5709002EBF0D083D08222124E321218BD
:104EB0006822D083D08222124E32124E8D1220D818
:104EC000C082C083753D01782EE2540F70E408E281
:104ED000540F70DE08E2540FC4F5F008E2540F4599
:104EE000F0F58308E2540FC4F5F008E2540F45F0E2
:104EF000F582C26D78A47900C3E5829410F582E54D
:104F0000839427F58340030980EEE5822410F5821F
:104F1000E5833427F583E96004D26DF6087900C390
:104F2000E58294E8F582E5839403F58340030980E4
:104F3000EEE58224E8F582E5833403F583E9206D0C
:104F4000046004D26DF6087900C3E5829464F582AA
:104F5000E5839400F58340030980EEE5822464F53F
:104F600082E5833400F583E9206D046004D26DF698
:104F700008E58275F00A84206D026002F608E5F00B
:104F8000F6E8245DF53DD083D0822279A47700092C
:104F900075F00577FF09D5F0FA22124E32124E8DC8
:104FA000124F8B75F008E571B42204782E8013B48B
:104FB0002A047830800CB4420478368005782E7547
:104FC000F006753D06E2540F700608D5F0F780092B
:104FD00079A4E2F70809D5F0F922124F9A12192A9A
:104FE00022124EB712192A227865E2700302509DF0
:104FF00024FD4038C082C0831200E41250F9D083EF
:10500000D08220521620510B305036121868703161
:1050100002509D12192A702902509D784DE2B583E5
:105020002008E2B5821B658270178071E224E2409D
:1050300070C082C0831200E41278F1D083D0825015
:105040000302509F7865E2B40F0C124FDA604E12E3
:105050004EAB604980EBB41007124FE1603F80E136
:1050600075F00384E5F0B40007124FDA70D3802D99
:10507000B40107124EAB70C98023B4021EC082C0B7
:1050800083124DA9E5828583F0D083D08240B2653A
:105090008270AEE5F0658370A8800280A4C322D33D
:1050A00022C082C0831200E4127947D083D082509C
:1050B00002D3227865E275F00384E5F0B4000A12A9
:1050C000514D12192A70EA802CB4010A125175123E
:1050D000186870DD801FB4021EC082C08312517830
:1050E000E5828583F0D083D08240C6658270C2E5B8
:1050F000F0658370BCC32280B8754832D25B3054EF
:1051000009C254C07412027AD074E548D36018C240
:1051100052C251C250121F3550E41239A620520615
:105120002051033050D8C3C0D0A8747405B802020F
:105130007404D0D0400512395D800312398322E512
:1051400082B4E807E583B40F02D322C322124E1EB5
:105150005002D322782EE260F9F5F008753D06E2A0
:10516000540F700608D5F0F7800979A4E2F7080912
:10517000D5F0F9C322027A69124E1E5004D322C31D
:1051800022782EE20860F6B40108E2F58275830009
:1051900080EDB40212E275F00AA4F58208E22582DD
:1051A000F58275830080D8B40320E275F00AA4F577
:1051B0008208E2258275F00AA4F58285F08308E270
:1051C0002582F58250B9058380B5B40405782F0295
:1051D0004DD1C39404F5F0782F024DC8B263B26488
:1051E0007551071237BD1237D3B264B2637518C058
:1051F000751900751A0C120A2230660C7518B075F4
:105200001900751A00120A22124AA0751810856535
:105210001985661A120A2222E53DB4031C78A4E619
:10522000B40A1608E624F6401008E624F6400A18E8
:10523000E675F00AA40826C322D32212521850039E
:1052400002461278ADF20252981274451282EDC2F3
:1052500045C2482252EF5311534D5379539053A7EF
:1052600053BE53D553E453F354025411544854736A
:10527000547B548D549C54D8552A554D55645585AE
:1052800055A155BD55C955E55601560D56295645EA
:105290005651566A52C352C378ADE224E0402412FC
:1052A00057B3401378ADE225E00490525493C0E028
:1052B000E225E093C0E02202586B12586A1200D730
:1052C000024AD8740A02586BD2A1C258C2A4D2575B
:1052D0001258691200E41220F8205102D322E53D51
:1052E000B402F978A4E624F640F208E624F6221285
:1052F00058681252C8401578A4E62430F51E08E616
:105300002430F51F12184212662A80AE742002580B
:105310006B125868125752402F12772C78A4E6C4AB
:105320000846F5F078A8E65403030345F07885F6BF
:1053300078A6E6C40846F5F078A9E6C42345F078D7
:1053400086F61276DE0252BA741E02586B12586844
:10535000125703401F12772C78A4E6C408467884BD
:10536000F678A6E6C408467883F6E47882F61276E4
:10537000DE0252BA741F02586B12586812584C75EC
:1053800018C0751900751A0F120A22D25F0252BA9C
:1053900012586812584C7518C0751900751A1012F9
:1053A0000A22C25F0252BA12586812584C7518C0CD
:1053B000751900751A51120A22D2610252BA125896
:1053C0006812584C7518C0751900751A52120A22C5
:1053D000C2610252BA12586812584C751A1B122137
:1053E000D30252BA12586812584C751A1B1221EC8B
:1053F0000252BA12586812584C751A1B1222140223
:1054000052BA12586812584C751A1B1221FB0252DC
:10541000BA125868123254402A12584C127445126B
:1054200082EDC245C248C243784DE2F58308E2F5F9
:105430008275186085831985821A120A22757F0386
:105440000252BA741602586B12586812325440F362
:1054500012584C127445D243784DE2F58308E2F5B8
:105460008275187085831985821A120A22757F0346
:105470000252BA12586820439880CD1258681258C8
:105480004C75F0C8128247D5F0FA0273C212586800
:1054900012584C751A1B1222A90252BA12586820CF
:1054A000150D1256CB402C12587E402778AEF2785C
:1054B000AEE2F552F55312584C7518C085521A7564
:1054C0001903301503751902120A220252BA74190F
:1054D00002586B741A02586B12586820150D125638
:1054E000CB40F012587E40EB78AEF278AEE2F55247
:1054F00012584C7518C085521A7519063015037567
:105500001905120A221268731268AA124B71D2A2EC
:10551000C259C2A1D2581200E41220F874182050C7
:10552000062051033052AE0244DB12586830742D0D
:1055300078B3E278B4F212584C7518C07519097432
:105540001B543F4480F51A120A220252BA125868BC
:1055500030740A1256CB500A741C02586B741D0228
:10556000586B70CF1258683074F3E478B4F2125864
:105570004C7518C0751909741B543F4440F51A1234
:105580000A220252BA1258687400127D6D7518C052
:1055900075190A741B543F4400F51A120A2202526C
:1055A000BA1258687400127D997518C075190A747A
:1055B0001B543F4480F51A120A220252BA1258684C
:1055C0007400127DB640DD80BF1258687402127DEF
:1055D0006D7518C075190C741B543F4400F51A12F0
:1055E0000A220252BA1258687402127D997518C0C4
:1055F00075190C741B543F4440F51A120A220252CA
:10560000BA1258687402127DB640DD80BF12586825
:105610007403127D6D7518C075190C741B543F44CA
:1056200080F51A120A220252BA1258687403127DC7
:10563000997518C075190C741B543F44C0F51A12A3
:105640000A220252BA1258687403127DB640DD80F5
:10565000BF7404127D6D7518C075190B741B543F0F
:105660004440F51A120A220252BA1282ED7518C08D
:1056700075190B741B543F4480F51A120A2202520A
:10568000BAC2A1D258C2A4D257124B711200E4126E
:1056900020F820520820501C205129D322784DE2B6
:1056A000F58308E2F582120102300806124D15203A
:1056B000E2E9C322121A8A70E2784DE583F208E526
:1056C00082F280E2121B6370D280EED2A1C258C275
:1056D000A4D2571258691200E41220F8205102D3C4
:1056E00022E53D60FA24FC40F6A93D78A47A00EA60
:1056F00075F00AA42640E8C5F070E4AAF008D9EFD6
:10570000EAC322D2A1C258C2A4D2571258691200C9
:10571000E41220F8205102D322E53DB404F9F5F05B
:1057200078A4E624F640F008D5F0F778A4E675F002
:105730000AA4082624E8402E78A6E675F00AA408F4
:105740002624C4402122E0E2E0E1E0E1E0E0E1E003
:10575000E1E0D2A1C258C2A4D2571258691200E4A3
:105760001220F8205102D322E53DB406F9F5F07875
:10577000A4E624F640F008D5F0F778A6E675F00A1E
:10578000A4082660E1C0E024F3D0E040D99057455A
:1057900093F978A4E675F00AA4082660C9C0E02948
:1057A000D0E040C278A8E624F640BB78A9E624F908
:1057B00040B42230087C784D740FF20874E9F2206E
:1057C000157C78ADE22400F5827583D07401F974FC
:1057D00080F875300185833185823212049B788090
:1057E000E6120158506278ADE22400F5827583D14B
:1057F0007401F97480F87530018583318582321225
:10580000049B7880E61201A8503678ADE22400F5BA
:10581000827583CF7401F97480F875300185833106
:1058200085823212049B7880E620630C20E01530DC
:10583000E10C125681740D2220E20920E3F4C32208
:10584000740E8006740C8002740BD322201518127B
:1058500037E9784DE2F58308E2F5827518E0858333
:105860001985821A120A2222222222C0E0126B21FA
:10587000125868D0E012674E1200AB024AD8C052EC
:10588000C082C083F5521267D1D083D082E552D056
:1058900052B322C5382538C53822E54A24E94008E4
:1058A000D2A3C256D2A2C2593098EFC298E599123B
:1058B0005893223099FDC299F59912589322C2A3A8
:1058C000C256C2A2C259C2B675380074051258B386
:1058D000E51E1258B3E51F1258B3221282771282C6
:1058E000771282771258BEE5371258B3E53812584E
:1058F000B33099FD221209900258FE12092CC0E023
:105900001258BEE5371258B3D0E01258B3E538123A
:1059100058B33099FD221282771258BEE5371258DB
:10592000B37980E71258B309DDF9E5381258B3307E
:1059300099FD22D216754A19751A001282EDE539C1
:10594000600B54F87007C227A227B392A5E53A600E
:105950000B54F87007C228A228B392A6E53B600B4F
:1059600054F87007C22CA22CB39280126DCEC28E56
:10597000C28CC2ADC2ABC2ACC2AF7581D5905988E2
:10598000C082C08375D00032D2AFD28C1271F4C203
:10599000ACD2991258DBB2B5754A19D2980259C5E2
:1059A000B40922F53812589AB51E2712589AB51F15
:1059B0002112589AB4461B12589AAF3812589A6F4F
:1059C00070101258DBD2B6D2A3C256D2A2C259125C
:1059D000589AB40ACBF53812589AB51EF512589A4F
:1059E000B51FEF12589AF537B46D03025A7BB46EA7
:1059F00003025A94B46F03025ACBB47003025B18CB
:105A0000B47103025B2CB47303025B3DB4740302F4
:105A10005B3FB47503025B53B47603025B6BB477F0
:105A200003025B6EB47803025B82B47903025BA36A
:105A3000B47A03025BBFB46C03025BD3B46B0302A2
:105A40005BF5B46A03025C30B46903025C4CB46871
:105A500003025CABB46703025CC3B46603025CDEA2
:105A6000B46503025DA2B464030264E6B463030296
:105A700064ADB461030265410259C5AF3812589A4A
:105A80006F70F51258DBD2B675F01E128247D5F052
:105A9000FA0273C212589AFD1424E0402B12589A4D
:105AA0002400FC7B0012589AFEAF3812589A6F708F
:105AB000178EF0EDF97480F88B308C3185F032124E
:105AC000049B125916754A190259C512589AFD14A9
:105AD00054E070F412589A2400FC247140EA7B02CE
:105AE00012589AFEEDFA788012589AF608DAF9AF51
:105AF0003812589A6F70D1C2A3C256C2A2C2598E30
:105B0000F0EDF97480F88B308C3185F0321203F0AF
:105B10001258E4754A1980B0AF3812589A6F70A8BD
:105B20001207501258DB754A190259C5AF3812587E
:105B30009A6F70091258FB754A190259C58089126B
:105B4000589AFD1424E0403712589A2400FC7B0137
:105B5000025AA512589AFD1454E0702312589A2440
:105B600000FC242540197B03025AE0025AC8AF38D2
:105B700012589A6F70091258F5754A190259C502E0
:105B80005AC879187D0712589AF309DDFCAF38120C
:105B9000589A6F70EA12675040E51276DE1258E4A8
:105BA0000259C5AF3812589A6F70D412772C1282EE
:105BB000771258BEE5371258B31202C80259C5AF62
:105BC0003812589A6F7066120D2E1258DB754A19EA
:105BD0000259C512589AFE12589AFD12589AFCAFF3
:105BE0003812589A6F70461206B640411258DB754B
:105BF0004A190259C512589AFE12589AFDAF381226
:105C0000589A6F702812068712827712827712587C
:105C1000BEE5371258B3EE1258B3ED1258B3EC127A
:105C200058B3E5381258B33099FD0259C5025AC825
:105C3000AF3812589A6F70F5128277128277125825
:105C4000BEE5371258B31211090259C5AF381258C0
:105C50009A6F70D912092460027401C0E012098899
:105C600060027402D0F045F0700A12079B1214A073
:105C7000120D2EE4C0E01258BEE5371258B3D0E042
:105C8000C0E01258B3E5381258B375F003128247DA
:105C9000D5F0FA1258BEE5371258B3D0E01258B317
:105CA000E5381258B33099FD0259C512589AFD14BF
:105CB00054E0702712589A2400FC2471401D7B0088
:105CC000025AE012589AFD1454E0700F12589A24A8
:105CD00000FC242540057B01025AE0025AC8AF3877
:105CE00012589A6F70F51282771282771258BEE5B9
:105CF000371258B374021258B3744E1258B37480EA
:105D00001258B374481258B374331258B374001253
:105D100058B3748D1258B374201258B374DA1258F1
:105D2000B374001258B3740F1258B374A01258B35E
:105D300074801258B374001258B374001258B374BC
:105D4000201258B374001258B374001258B3740080
:105D50001258B374001258B374001258B37400127E
:105D600058B374001258B374001258B37400125828
:105D7000B374001258B374001258B374001258B3BD
:105D800074001258B374001258B374001258B374EC
:105D9000001258B3E5381258B33099FD0259C502C4
:105DA0005AC812589AF58312589AF5822460E583EE
:105DB00034F040EB12602E12589AFD1454E070DF5C
:105DC000780075F02074FFF208D5F0FB78001258C7
:105DD0009AF208DDF9AF3812589A6F70C21258DB88
:105DE00075F005128247D5F0FA1258E4751A0130A1
:105DF00008AD12606412604A12603C1219A07898D3
:105E000079007A0A75F00FE3540FF652F00809DAB8
:105E1000F643F0F0E5F00478A179847A0512187B56
:105E2000600B125EC35006751A04025D9F12604A31
:105E300012603C1219A078A4790A7A0675F00FE373
:105E4000540FF652F00809DAF643F0F0E5F0047862
:105E5000A979877A0312187B600B125F615006756F
:105E60001A06025D9F12604A1260AD751A650259EA
:105E7000C5C0E07828E583F208E582F2D0E022C0D0
:105E8000E0782AE583F208E582F2D0E022C0E078EB
:105E900028E2F58308E2F582D0E022C0E0782AE229
:105EA000F58308E2F582D0E022E5822400F582E560
:105EB00083341BF58322E5822400F582E583343B9D
:105EC000F5832212603CAB83AC82901B00C08379C7
:105ED000007530038583317532009000561203A59A
:105EE0001205161203A51205749000567A80E0A3DD
:105EF000F5F0E0A36C7005E5F06B6017DAF0D08385
:105F00000583740024C0E58334C550C17405126054
:105F100010D322D083EA2AF5F0E4C395F0F582127B
:105F20005E71789879007A0A75F00FE3540FF65293
:105F3000F00809DAF643F0F0E5F004600C121A8D6F
:105F4000700A7406126010D322121A8DE58225821F
:105F5000F582E5833583F583125EA9125E7F0262C6
:105F6000B512603CAB83AC82903B00C08379007576
:105F700030038583317532009000561203A5120557
:105F8000161203A51205749000567A80E0A3F5F06E
:105F9000E0A36C7005E5F06B6017DAF0D083058341
:105FA000740024C0E58334A550C17405126010D379
:105FB00022D083EA2AF5F0E4C395F0F582125E71EF
:105FC00078A4790A7A0675F00FE3540FF652F008B8
:105FD00009DAF643F0F0E5F004601D121B73701B44
:105FE000AB83AC8212603CEBB58306ECB58202C396
:105FF000227404126010D322121B73E5822582F5ED
:1060000082E5833583F583125EB6125E7F0262B548
:10601000F51A22C082C083E58312674FD083D082F5
:10602000C082C083E58212674FD083D08222C0E055
:10603000782CE583F208E582F2D0E022C0E0782CEB
:10604000E2F58308E2F582D0E02274001258B374BE
:10605000001258B374001258B374001258B374008D
:106060001258B32275831B75821B75F040C0F0C0B7
:1060700082C0837530018583317532001203A51209
:106080000516D083D082C082C083753003858231EB
:106090007532001203A51205DCD083D0820583057A
:1060A00082D0F0D5F0C77533FF7534FF227401F943
:1060B0007418F875300075310075320012049B7445
:1060C00001F97419F87530017531D97532FF120470
:1060D0009BAC1812603CE5822420F582E583347D78
:1060E000F583C082C0837401F9743CF87530008573
:1060F000833185823212049BD083D0827401F9747B
:1061000010F87530008583318582321203BF781014
:10611000E2F5F0E518253CC395F0F51812603C1245
:106120004CB778537980E2F72519F5190809E2F799
:106130002519F51978167953E2F3FA0809E2F32ADA
:10614000FAC3E5199AF51912603C124CE112603C51
:10615000E58275F008A42420F582500205F0A8F02D
:10616000E58375F008A4282400F5837408F9748089
:10617000F875300085833185823212049B7880E582
:10618000187A082608DAFCF518789879007A0A75E2
:10619000F00FE3540FF652F00809DAF643F0F0E599
:1061A000F0041266EC78A4790A7A0675F00FE354CD
:1061B0000FF652F00809DAF643F0F0E5F004126643
:1061C000F47408F97480F875300085833185823263
:1061D0001203F07880E5187A08C39608DAFBF51800
:1061E00012603CC3E58233F582E58333F583C3E572
:1061F0008233F582E58333F583E5822400F582E579
:1062000083245BF583C082C0837404F97480F875BD
:10621000300185833185823212049BD083D0827411
:1062200004F97412F87530018583318582321203C6
:10623000BF78807912E5197A0426F5F0E3C5F0C33A
:1062400095F00809DAF3F5197401F97418F8753046
:10625000007531007532001203F07401F97419F8F9
:106260007530017531D97532FF1203F075831B75D6
:10627000821B75F040C0F0C082C0837530038583F7
:10628000317532001203A5120516D083D082C08268
:10629000C0837530018582317532001203A5120565
:1062A000DCD083D08205830582D0F0D5F0C775336A
:1062B000FF7534FF22125E9BE5828583F0125E8DAE
:1062C000C39582C0E0E5F09583D0F045F07002C33D
:1062D0002250030263D0125E9BC0E0C3E58224FE1D
:1062E000F582E58334FFF583D0E0125E7FE5828599
:1062F00083F0125E8DB58207E5F0B58302C32212EA
:106300005E8DAF83125E9BEFB58310AE8290002C42
:106310007880E0F6A308E0F60263337EFE8F830503
:10632000837402F97480F875300385833175320007
:1063300012049B79007530038F317532009000563E
:106340001203A51205161203A51205748F83758218
:1063500000125E8D7D00E5836F7002AD82ED2456E4
:10636000F58275830050020583C3EE9D20E05A0339
:10637000FCC082C083A3A3E0FAA3E0FBD083D08259
:10638000EAF0A3EBF0A3DCE9EE2456F58275830076
:10639000500205837880E6F0A308E6F079007530B6
:1063A000038F317532009000561203A51205C812F2
:1063B00003A51205DC853033853134125E9BEFB5C1
:1063C00083030264A40F0263047408126010D322D2
:1063D000125E8DAF83125E9BEFB58310AE8290008C
:1063E0002C7880E0F6A308E0F60264047E008F8338
:1063F00015837402F97480F8753003858331753222
:10640000FE12049B79007530038F317532009000C5
:10641000561203A51205161203A5120574125E8DFD
:106420007DFEE5836F7002AD82ED2456F5827583A3
:106430000050020583C3ED9E20E06B03FCC0E0C367
:10644000E58224FEF582E58334FFF583D0E0C08247
:10645000C083E0FAA3E0FBA3EAF0A3EBF0D083D083
:1064600082DCDAEE2456F5827583005002058378CB
:1064700080E6F0A308E6F079007530038F317532BD
:10648000009000561203A51205C81203A51205DCE0
:10649000853033853134125E9BEFB583030264A4EB
:1064A0001F0263D5C3227409126010D32212589AB6
:1064B000F58312589AF58212589A702712589A70DA
:1064C00022AF3812589A6F701AC01EC01F85831EE3
:1064D00085821F12184212662AD01FD01E1258DB66
:1064E0000259C5025AC812589AF58312589AF58271
:1064F000AF3812589A6F70EBC01EC01F85831E857F
:10650000821F1218427401F97480F87530007531D9
:106510000075320012049B7880E6C3951EC3951F58
:10652000D01FD01E251E251FF67401F97480F87542
:1065300030007531007532001203F01258DB025939
:10654000C512589AF583AF3812589A6F7095128217
:10655000771282771282771258BEE5371258B374D9
:10656000001258B3E51A1258B374001258B37400ED
:106570001258B374001258B374001258B3E53812AD
:1065800058B33099FD0259C5906590C082C08332DE
:106590007581D575D0000273C2C082C083E58224A4
:1065A00020F582E583347DF5837401F9743CF87538
:1065B00030008583318582321203F0D083D082C0CF
:1065C00082C083E58275F008A42420F5825002057C
:1065D000F0A8F0E58375F008A4282400F58374047E
:1065E000F97480F87530008583318582321203F0AA
:1065F000A3A3A3A37404F97484F8753000858331D0
:106600008582321203F0D083D082E5824583600E0A
:10661000E5822418E58334FC74FFF5F0500BC0824A
:10662000C083124CE1D083D0822212092CC0E074C6
:1066300001F97480F875300075310075320012046C
:106640009B7880E6D0F0C395F0F67401F97480F879
:106650007530007531007532001203F022753C0070
:106660007854E4F2788075F00876FF08D5F0FA22C5
:10667000751E30751F30C263C26475F005C0F0D25C
:10668000A3C256C2A2D259D2A1C258D2A4C2571292
:10669000665D1220F8D0F0205009205106D5F0DDBB
:1066A0000266E712670C403F1200D77885E6B4FF18
:1066B00005C32275F005C0F01220F8D0F020510675
:1066C000D5F0F30266E7E53DB4021C78A4E624F6B3
:1066D000401508E624F6400F78A4E62430F51E089D
:1066E000E62430F51FC3221200ABD32278987980BC
:1066F0007A05800678A479857A03E608540FC4F5F4
:10670000F0E608540F45F0F709DAEF222050313057
:10671000513AE53D600624FD24FC40301266F41237
:1067200000E475F005C0F01220F4D0F020501120E4
:106730004406D5F0F002674C1211BAB40B0E800378
:106740001266EC753C007854E4F2C322D322222274
:10675000781DE254C07078E275F00A84C445F07880
:1067600082F6781CE254C07066E275F00A84C44573
:10677000F07883F6781BE254E07054E275F00A84F6
:10678000C445F07884F6781AE2604454E07040E240
:1067900075F00A84C445F0C0E07818E2030354C0E1
:1067A000D0F045F07885F67819E2602354F0701F38
:1067B000E275F00A84C445F0C0E0781EE254F87037
:1067C0000EE2C42354E0D0F045F07886F6C322D31D
:1067D0002290000075F019C0F07402F97480F87509
:1067E000300185833185823212049B7881B6FF02A5
:1067F000801318E55230080AB4FF0788F07855E294
:10680000A8F0666011E5822410F58250020583D05D
:10681000F0D5F0C3C322D0F0A3D32230084DE582D7
:1068200024FFF582E58334FFF58375F019E58224B2
:1068300080E58334FE5005900000800AE582241034
:10684000F58250020583C0F07402F97480F8753047
:106850000185833185823212049B7881B6FF0280E4
:106860000518E6B55207D0F0D5F0C2C322D0F0A388
:10687000D32222300F0CC20F12675040051276DE71
:10688000800312772C7885E6C45403E6540F78868B
:10689000E6C45401E6540F7884E6C4540FE6540F5E
:1068A0007883E6C4540FE6540F2230080A1267D1E9
:1068B0005005126872800312692322C2AC1271F46F
:1068C000C2AC128277128277D299C2B674FF125884
:1068D000B375380074421258B374621258B3741509
:1068E0001258B3742A1258B3741B1258B37400129E
:1068F00058B374001258B374001258B3740012588D
:10690000B31202D575F010C0F074001258B3D0F075
:10691000D5F0F4E5381258B33099FDC24FD2B61213
:1069200071F42222201401227475787A12012F50FA
:106930001A206819D268126E4B7518C075190B743D
:106940001A543F4400F51A120A2222C26812772C08
:10695000203304203433227884E6543FF5F07970F4
:10696000E365F0702109E3788366701A203516D24A
:1069700035126E4B7518C075190B741A543F4400CC
:10698000F51A120A222230342F7884E6543FF5F0AB
:106990007972E365F0702109E3788366701A203517
:1069A00016D235126E4B7518C075190B741A543FF8
:1069B0004400F51A120A2222C23522C2AC120A6021
:1069C000600CF5188819120DA1120A7880EFD2AC6C
:1069D000227E007F8490000075F000E49325F0F59E
:1069E000F0A3C3E5829EE5839F40F0E5F0700222AC
:1069F00000E5F0C0E0E58312674FE58212674FD0F3
:106A0000E012674FC2ADC2ACD216D2A3C256D2A218
:106A1000C259C2A1C258D2A4C257C2A080EC75F01C
:106A2000641205EF20E50430E30122C2AFB2B512D3
:106A3000825FB2B512825FD5F0E712035880FB2265
:106A400030083C7400788A12013E40337F087E0093
:106A50007478787A12012FCE13CE05E0DFF4201778
:106A60000E7400789A12013E5005EE655460108E47
:106A7000548E527518C075190485521A120A2222B2
:106A8000C2AF75181075190FF51A120A22D2AF226B
:106A9000223008FC205CF97401788A12013E40F033
:106AA0007477787A12012FE492E0C0E07476787AF5
:106AB00012012FD0E033FE20170E7401789A1201D4
:106AC0003E5005EE655560C88E55EE20E10630E07B
:106AD00028026B0C30E014A25E725D50B3C25EC23D
:106AE0005D126DAD74F8126A8080A5D25EC25D122F
:106AF0006DAD74F7126A808097205D0ED25DC25E24
:106B0000126DADD25B74F6126A808084A226825D1B
:106B100040F8D25DC25E126DC174F5126A80026ADD
:106B200090C082C083D083D0822222304309C2A386
:106B3000C256D2A4C25722D2A3C256C2A4C257225E
:106B400020080122300819C0E0C082C083740712F7
:106B50000188D083D082D0E04003026B7E026B605C
:106B6000201708206033D260205F2ED25FD260757C
:106B700018C0751900751A0F120A22026B99201796
:106B800008306015C260305F10C25FC2607518C007
:106B9000751900751A10120A22300819C0E0C08257
:106BA000C083740F120188D083D082D0E0400302EA
:106BB0006BD3026BB5201708206233D26220612E9E
:106BC000D261D2627518C0751900751A51120A2265
:106BD000026BEE201708306215C262306110C2618C
:106BE000C2627518C0751900751A52120A2222C2A3
:106BF000B675380074031258B3E51E1258B3E51F7A
:106C00001258B3744E1258B374081258B374011268
:106C100058B374061258B37848E2F5F0E5F012580C
:106C2000B308E2F5F0E5F01258B3784AE2F5F0E582
:106C3000F01258B308E2F5F0E5F01258B32442F828
:106C4000E2784CE2547FF5F07844E2C36001D3E58A
:106C5000F092E7F5F0E5F01258B375F000E5F012A8
:106C600058B3E5381258B33099FD22C2B6127C35BC
:106C7000127BC475380074031258B3E51E1258B362
:106C8000E51F1258B3744E1258B3740C1258B374F3
:106C9000001258B3740A1258B3C082C083A3A3A3CE
:106CA000E49375F064A4C0E0E5F01258B3D0E012AC
:106CB00058B3A3A3A3A3E49375F064A4C0E0E5F0E4
:106CC0001258B3D0E01258B3D083D082E493125854
:106CD000B3A3E4931258B3A3A3A3E4931258B3A3AA
:106CE000E4931258B3E58D1258B3E58B1258B3E50F
:106CF000381258B33099FD22C2B6121254C0E07552
:106D0000380074031258B3E51E1258B3E51F125829
:106D1000B3744E1258B374041258B374021258B3B9
:106D200074021258B3E57D1258B3D0F0E5F0125852
:106D3000B3E5381258B33099FD22C2B61211D4C04F
:106D4000E075380074031258B3E51E1258B3E51FFE
:106D50001258B3744E1258B374041258B37402121A
:106D600058B374021258B3E57D1258B3D0F0E5F071
:106D70001258B3E5381258B33099FD22C0F088F0AC
:106D8000C0F0C2AF7575007850E2F54CF5F008E23E
:106D9000F54DD2AF45F0D0F0A8F0D0F07009B22692
:106DA000202604126DB722D22675750322C2AF7554
:106DB0004CFF754DFFD2AF757500C209C226D2A730
:106DC00022126D7CD25BD25522C26E0281A7D26E96
:106DD0000281A7305D1220260F543F4400F51A753A
:106DE00019087518C0120A2222D2B2C2B4D293C3B3
:106DF00022D2B2C2B4D29312825F20B2ECC29312FA
:106E0000825F30B2E4D29312825F12825F20B2D9E5
:106E1000C29312825F12825F30B2CED2B2C2B4D2BB
:106E200093D3221204E6C2847454120500E41204BF
:106E3000C01204D3F5F06448255E33F55EE5F02515
:106E40005FB2E003F55FD9E9D284227583DD75F086
:106E500010753003858331753200C083C0F0120392
:106E6000A51208BED0F0D0830583D5F0E47533FFBA
:106E70007534FF75760075770022E5822400C0E046
:106E8000E58334DDF8D0E0C322C082C0837401F909
:106E90007480F875300385833185823212049B78C3
:106EA00080B6020CE57724FFF577E57634FFF576BA
:106EB000D083D08222126E7AC082C083F58288830A
:106EC000126E89788076007401F97480F875300349
:106ED0008583318582321203F0D083D08222126EF4
:106EE0007AC082C083F5828883C082C0837401F92E
:106EF0007480F875300385833185823212049B7863
:106F000080B60209D083D082D083D08222E5772454
:106F100001F57750020576D083D0827880760274AE
:106F200001F97480F875300385833185823212034C
:106F3000F0D083D08222126E7A126E7AC082C08321
:106F4000F5828883126E89788076017401F97480E5
:106F5000F87530038583318582321203F0D083D0F7
:106F60008222126E7AC082C083F5828883126E8973
:106F7000788076037401F97480F875300385833165
:106F80008582321203F0D083D08222126E7AC082C0
:106F9000C083F58288837401F97480F875300385A5
:106FA000833185823212049B7880E6B40102800C22
:106FB000B402028007B4030280027400D083D0823E
:106FC000221204E6C2847454120500E41204C012B2
:106FD00004D3B40205755E018002D9F3D284227510
:106FE0005E007583DD75F00F753003858331753272
:106FF00000C083C0F01203A51205161203A5790084
:10700000126FC1D0F0D0830583E55E7026D5F0D82D
:107010007530038583317532001203A512051612EF
:1070200003A579A0126FC17533FF7534FFE55E705B
:1070300002D322C322E577457660167867E2F5F041
:1070400008E245F0600BD37868E2957718E2957610
:1070500022C322126F8BC2B675380074031258B364
:10706000E51E1258B3E51F1258B374501258B3748A
:107070007D1258B3900000E536600F9003E814606D
:10708000099007D0146003900BB87E7D7F0875F0DF
:1070900000C0F0126F8BB40203D38001C3D0E03381
:1070A000F5F0A3DFEC1258B3DEE2E5381258B33046
:1070B00099FD22C28C758A45758C5DD28CB20020F8
:1070C000000132C000C001C0D0C0E0C0F075D008DF
:1070D000D2541211B91271D5051DE51D20E00C2006
:1070E000E10930161AE51D541F6059201604E54BBE
:1070F0006002B2B5D0F0D0E0D0D0D001D0003220C4
:107100005905A226B392A2E51D30E203127F03E5E2
:107110001D541F7032D255C27278ABE2D5E006D250
:1071200071D272743CF2C082C083127DD6D083D0FB
:1071300082E4B54748B5495AB56362B56E63B57E1A
:1071400067B57F68B54A69E4B54B43B54871B54545
:1071500072B54E76B57577E54D454C601DE54D240D
:1071600001F54D5002054C454C700FC209205C0AD8
:10717000205D07126DB7D25BD2550270EBD547B5D3
:10718000C2097549B4757C00D247D24A80A7154B15
:1071900080B9D549A3C245C246C247809B156380CA
:1071A0009AD56E9AC2708096157E8095157F8094D0
:1071B000D54A947546033016030265880271381566
:1071C00048808BD5458BD24E8087154E8086D575ED
:1071D00086C2A78082E51DA2E330560292A33059F1
:1071E0000292A230580292A122C2B6204F02D2B619
:1071F0001271F43275C800C2ADC2AC75CBFF75CA4E
:107200009875CDFF75CC98759853C298C299D2AC39
:10721000C2BC75C8347599062275C800C2ACC2AD2F
:1072200075980075CC2B75CDEBD2AD75C804227561
:10723000C800C2ACC2AD759800E58A242BF5CC54C9
:107240000F658C24EBF5CDD2AD75C80422C2A8C25F
:10725000AAC289C28BC2ACC2A9C2AB758F0112058A
:10726000FCD216126DCE126DADE4F53C7854F27876
:107270007A75F010F2D5F0FCC25CC25DC25EC25FEE
:10728000C261753EFF7540FF751D04C244C245C210
:1072900046C247754901754A00C24AD25475720008
:1072A000C235C218C219D24EC24F754510E4F5411D
:1072B000F542F543F535F537121E71751E00751F41
:1072C00080E4F547F550F54FF558F559F53FC223E1
:1072D000C224C225C22B7437785AF2785BF2785CEC
:1072E000F2785DF2D21F75460375480178AC7A05D5
:1072F00076FF08DAFBC20F7818E47A07F208DAFCA6
:10730000C2107552FF855254C211C208757E0375B2
:10731000631E756400C267C20DC20EC209C20AC2F2
:107320000BC263C26475610075600075F006784237
:10733000E4F208D5F0FB7948E4F309F3794AF3095C
:10734000F3784CE4F21213C8754BFAB2B57533FFFB
:107350007534FFD268756D007827740AF2127C14B8
:10736000C270756E0175711AC201C202C203C204F5
:10737000C205D2A075750075760075770078AA747D
:10738000FAF2E478B2F278B3F278B4F278AB743C03
:10739000F2C274C273C26F757C00127D49C275D28D
:1073A00076C277758901758A3E758C5DC2B9D2A99E
:1073B000D28CD2B61271F4D2AFD293C2B4D2B2B2DE
:1073C000B522C21675510375F003128247D5F0FA43
:1073D000C263C26412364375510375F003128247CB
:1073E000D5F0FAC263C2641234E2C2AF02000020D8
:1073F000051320040820020D200102C3221213DC11
:1074000012781FD322127928D32275F000C0F0120F
:107410002300D0F0500343F008E5F022307314202D
:10742000432278B4E2307106C271600214F224FA89
:1074300050092230740E78B4E27009E57B54017073
:10744000031200E422C274C273E478B4F222C2AF21
:10745000754BFAB2B512825FB2B512825FB2B5D285
:10746000A07581D575D00012724D126B211269D1B1
:10747000126E4B121CA0754BFA120C9F1273EF7513
:1074800051031237BD1237D31200F17518807519E8
:1074900004751A80120A22D21730080F120AF0124D
:1074A0006A40126A91126924126B40D2B7D2AFC2FD
:1074B00016C21700000020B70912825F20B703022E
:1074C0001CBA300832120AF012741CE5795420609C
:1074D0001178AAE2D5E00A12772C1268BB78AA7458
:1074E000FAF2E57C6002157C30080C126A40126AE0
:1074F00091126924126B40E5646003D5640E127D1D
:10750000421238B71268731268AA800CD2A3C2560E
:10751000C2A1D258D2A4C257E56370031269BBC29C
:1075200059D2A1C258126B2BC263C264D25B78607D
:10753000E2600D24FD40097574021239A61273EF42
:107540007861E2600D24FD40097574031239A612BA
:1075500073EFE5785440600620A80312332D122003
:10756000F8205108205005205202801A302F09308F
:107570004606126B2102757E1244CD1273EF7827F6
:10758000E215E0F2700878277414F20274AB02740A
:10759000E20074A2127626E8127661E91276611290
:1075A00076982274A2127626E8127661E712766146
:1075B00009D582F81276982274A2127626E81276FD
:1075C0006174A3127626127681F709D582041276A9
:1075D0009822C296D297000000C29780E974A21246
:1075E0007626E81276611275EA2274A312762612C4
:1075F0007681F91276982274A27A08C29600000069
:10760000C297335005D29602760CC296D2970000EC
:1076100000C297DAEDD29600D297000000309604AF
:10762000C297C322D3227A08D296D29700000000D4
:10763000000000000000000000000000C2960000F2
:1076400000C297335005D29602764DC296D297006B
:107650000000C297DAEDD29600D297000000C297E0
:10766000227A08335005D29602766DC296D29700E0
:107670000000C297DAEDD29600D297000000C297C0
:10768000227A08D296C29700000000D297C33096A3
:1076900001B333DAF0C29722C296000000D29700FD
:1076A0000000D29622781079D1C0827582051275B9
:1076B000B8D08278D1B6870E08B6E00A08B633068D
:1076C00008B6A902C322D3221276A54001227882ED
:1076D0007600087600087600087601087601788042
:1076E00076000876007884E6543FF678007980C00A
:1076F000827582071275A3D082128247781479802E
:10770000C0827582071275A3D08212824778D17623
:10771000870876E00876330876A9781079D1C08298
:107720007582041275A3D082128247227802798270
:10773000C0827582051275B8D082227886E603C4AD
:10774000540775F018A4C0E07884E6C4540375F0BB
:107750000AA4F5F0E6540F25F0D0F025F075F03CC2
:10776000A4C0F0C0E07883E6C4540775F00AA4F51D
:10777000F0E6540F25F0D0F025F0F5F0D0E034001D
:10778000C5F022207556206921C0D0C0E0E8C0E0D5
:10779000C0F0E54E700385716F754E08D26C12789B
:1077A0009BD0F0D0E0F8D0E0D0D0C2893220692957
:1077B000C0D0C0E0E8C0E0C0F0E54E7003756F00D7
:1077C000754E08A2B2B3926C127980308502D20352
:1077D000D0F0D0E0F8D0E0D0D0C28B32C2A8C289BD
:1077E000322075C9206926C0D0C0E0E8C0E0C0F0F2
:1077F000E54E700385716F754E08C26C12789B3030
:107800008502D203D0F0D0E0F8D0E0D0D0C28B32E5
:10781000C2A8C2AAC293C2B4C0E0128247D0E0C2DA
:1078200075C293C2B4C289C28BD2B2D2B3C26975D7
:107830004E0085716FC203C2B8D288D2A8C2BAD234
:107840008AD2AA22C275C2A8C2AAC289C28B22E564
:1078500071141475F00884F5F0C0F0782EE230E071
:1078600002B26A30E102B26A30E202B26A30E30286
:10787000B26A08D5F0E7D0F0E230E002B26B30E156
:1078800002B26B30E202B26B30E302B26B08D5F0A9
:10789000E7206A05306B02C322D322E56FB571077A
:1078A000A26C926A0278E5B40107A26C926B02782E
:1078B000E5C3E57114956F403275F00484242EF809
:1078C000E205F0D5F006A26C92E38016D5F006A290
:1078D0006C92E2800DD5F006A26C92E18004A26C5D
:1078E00092E0540FF2D56F02D2692285716FD2698E
:1078F00022754832127810305405C25412027AE5CB
:107900004860113069F1E56F700A12784412784FBF
:107910004002C322127844D322C2A8C2AAC293C290
:10792000B4C0E0128247D0E0D275C293C2B4C2891B
:10793000C28BD2B2D2B3C269754E00756F00C2035A
:10794000C2BAD28AD2AA22754832127919305405A5
:10795000C25412027AE548600C3069F1E56F700597
:10796000127844C322127844D322C330E001B330EA
:10797000E101B330E201B330E301B330E401B322FB
:10798000E56F75F00584C0E024ECD0E04055242E6E
:10799000F8E2A26C92E503F2E56F700BE2541FB4BB
:1079A0000B40756F05803B056FE5F0B40434E212BF
:1079B000796A502F540FF218E2540FB40F24D3E811
:1079C000942E782EF20404C082F58275F00B08E242
:1079D00065F0F5F0D582F7D082540F7006D2697544
:1079E0006F00221279282201000000000000000030
:1079F000000A000000000000000000040600000073
:107A00000000000000080E0300000000000000005D
:107A1000010702000000000000000A060801000043
:107A2000000000000402040F00000000000008062F
:107A3000090809000000000000010E050F05000004
:107A40000000000A0C0A090B0300000000040E0BE2
:107A500000040502000000080E06070804070100E4
:107A6000000001050A040D080E75F00A79987700E8
:107A700009D5F0FA782EE2FA60400824F25007EABD
:107A800024F328F87A0DE2540FF26029EA1475F015
:107A90000AA424E7F58274003479F58379A17E0085
:107AA0007B0AE493F5F0E2A42E2775F01084FEA77C
:107AB000F0A319DBED08DACEC322D322094300A0DC
:107AC0000954009F0966009E0977009D0989009C62
:107AD000099B009B09AD009A09BF009909D2009843
:107AE00009E4009709F700960A0A00950A1D009418
:107AF0000A3000930A4300920A5700910A6B0090E3
:107B00000A7F008F0A93008E0AA7008D0ABB008CA3
:107B10000AD1008B0AE7008A0AFE00890B1400884C
:107B20000B2B00870B4300860B5C00850B750084D4
:107B30000B8E00830BA700820BC100810BDB008042
:107B40000BF6007F0C10007E0C2B007D0C47007C98
:107B50000C64007B0C81007A0C9E00790CBB0078D1
:107B60000CDB00770CFB00760D1B00750D3B0074E1
:107B70000D5B00730D7D00720D9F00710DC20070D2
:107B80000DE4006F0E07006E0E2C006D0E51006CA0
:107B90000E76006B0E9B006A0EC100690EE900684C
:107BA0000F1100670F3900660F6100650F890064CF
:107BB0000FB300630FDE0062100900611034006033
:107BC000105F005F7F42907ABCE493A3F5F0E493EA
:107BD000A3C3958BE5F0958D5015A3A3DFEBE5824C
:107BE00024FFF582E58334FFF583E49314800BA32F
:107BF000E493BF4205907ABC8010C0E0E58224F98E
:107C0000F582E58334FFF583D0E02290006BE0A29B
:107C10008733F02290006C7400F090006B7455F084
:107C200090006D74FFF090006F7405F090006E741A
:107C300012F0D28122D286A2A4C0D0D2A475F000C4
:107C4000D5F0FDD5F0FDC28E53890F438910758B99
:107C500000758D00C28FC2AFC2A4D28E20860330C1
:107C60008FFAC28E308F06758BFF758DFFD2AFD025
:107C7000D092A422F024FE4005308102C2812290DD
:107C8000006FE0D5E0EE7442F0127C35D281E58BD6
:107C90002499E58D34F24014E58B24E1E58D34F32D
:107CA000400EE58B24E0E58D34FC40087415800619
:107CB000741180027412FE90006EE06E6013EEF09C
:107CC000E5785404700B7518C07519008E1A120AE5
:107CD0002222127C0B603904603690006DE020E0B7
:107CE00010D2E0F090006CE070047405F022E4F033
:107CF0002290006CE0602C14F07028E5785402703B
:107D0000227518C0751900751A14120A22027D23F3
:107D100090006DE030E00DC2E0F090006CE070CEBD
:107D2000743CF02290006CE060F914F070F5E57896
:107D3000540270EF7518C0751900751A13120A22D3
:107D400080E1127C7F127CD2229002EC75F008E474
:107D5000F0A3D5F0FB9002F475F00874FFF0A3D502
:107D6000F0FB22C0E0127DB6D0E0B3502CC0E0247E
:107D7000F8D0E04022C082C083F5F024F4F582E41C
:107D80003402F583E0C5F024ECF582E43402F58397
:107D9000E5F0F0D083D082D322C0E024F8D0E040D8
:107DA00013C082C08324ECF582E43402F583E4F04E
:107DB000D083D082C322C0E024F8D0E04016C08235
:107DC000C08324ECF582E43402F583E0D083D082D2
:107DD0006002D322C3229002EC75F008E06003B485
:107DE000FF05A3D5F0F62220E70414F080F43072EA
:107DF000F114F0B480ECE4F080E8B44007740012B1
:107E00007DB6803DB441077401127DB68033B44223
:107E1000077402127DB68029B443077403127DB63D
:107E2000801FB444077404127DB68015C0E024E4BA
:107E3000D0E040132324B0C0E07400347EC0E022C0
:107E4000C3740122D380FAE4C322A243B380F2D2E6
:107E500055A26F80EC80F0A20980E6A20B80E2A21E
:107E60007780DE80DF80E0A20A80D63070D280D4B6
:107E7000E576457760CA80CC12703580C4A25E7208
:107E80005DB380BDA25D822680B7A25DB02680B1C1
:107E9000A25E80ADC330730920430678B4E270015E
:107EA000D3809EA26EB38099C3E57E6001D380919A
:107EB0008098809B80998097809580938091808F17
:107EC0008093809380958097809980998099809BFA
:107ED000809E80A480A780AC80B080B480B680C330
:107EE00080C68004800E8018C3204305E57F6001B2
:107EF000D3027E41C3304305E57F6001D3027E415A
:107F0000027E47127FFD300819C0E0C082C0837432
:107F100004120188D083D082D0E04003027F38026F
:107F20007F22E539B40D0A302102802CD221D38082
:107F300015127DFA6022800EE539B40D062021036A
:107F4000027F58C221C34009C227A227B392A5804D
:107F500007D227A227B392A5300819C0E0C082C07B
:107F6000837405120188D083D082D0E04003027F61
:107F70008A027F74E53AB40D0A302202802CD222A4
:107F8000D38015127DFA6022800EE53AB40D0620EA
:107F90002203027FAAC222C34009C228A228B392A8
:107FA000A68007D228A228B392A6300819C0E0C044
:107FB00082C083740B120188D083D082D0E040034A
:107FC000027FDC027FC6E53BB40D0A302A02802C1A
:107FD000D22AD38015127DFA6022800EE53BB40DC3
:107FE00006202A03027FFCC22AC34009C22CA22C0D
:107FF000B392808007D22CA22CB3928022B20C3094
:108000000C60E5795410600330431BE57A5404702A
:1080100003204538E57A54017003204611E57A546F
:10802000027003204717C26F755000028062E5504E
:10803000B401028024755001754F40801CE550B496
:1080400002028015755002754FA0800DE550B403F3
:10805000028006755003754FF0E54F23F54FA2E0FF
:10806000926F22C227A227B392A522D227A227B3BA
:1080700092A522B227A227B392A522F5F0030354BA
:108080003FB40258E53964086005E539B40D4AE5A6
:10809000F089F0C0F0300819C0E0C082C0837404D9
:1080A000120188D083D082D0E040030280C00280D9
:1080B000B1D0F0A9F05403B4020D1280630281A57F
:1080C000D0F0A9F00281A5B4010612806B0281A54F
:1080D000B403061280730281A50281A3B40362E592
:1080E0003A64086005E53AB40DEFE5F089F0C0F0B8
:1080F000300819C0E0C082C0837405120188D083A3
:10810000D082D0E0400302811F02810CD0F0A9F0A0
:108110005403B40211C228A228B392A60281A5D0AA
:10812000F0A9F00281A5B4010AD228A228B392A630
:108130000281A5B40309B228A228B392A680668062
:1081400062B4045FE53B64086005E53BB40D54E5AB
:10815000F089F0C0F0300819C0E0C082C083740B11
:10816000120188D083D082D0E04003028183028153
:1081700071D0F0A9F05403B4020FC22CA22CB39218
:10818000808022D0F0A9F0801CB40109D22CA22C4E
:10819000B392808010B40309B22CA22CB3928080D9
:1081A000048000D322C322C0E07417306E21B53999
:1081B00007C227A227B392A5B53A07C228A228B3BF
:1081C00092A6B53B07C22CA22CB39280D0E022B578
:1081D0003907D227A227B392A5B53A07D228A228F9
:1081E000B392A6B53B07D22CA22CB39280D0E0224A
:1081F000B4010775190F751AE122B4020775190F3A
:10820000751AE222B4030775190F751AE322B40434
:108210000775190F751AE422B4110775190F751A2D
:10822000D122B4120775190F751AD222B41307752B
:10823000190F751AD322B4140775190F751AD422A1
:1082400075190F751AD422C28E53890F4389107580
:108250008BD6758D97C28FD28E308FFDC28E22C283
:108260008E53890F438910758BEB758DCBC28FD2DE
:108270008E308FFDC28E22C28E53890F438910E546
:108280008AC4242BF58B758DEBC28FD28E308FFD77
:10829000C28E22543F4400F51A75190A7518C0029F
:1082A0000A22543F4480F51A75190A7518C0020A4B
:1082B00022543F4400F51A75190C7518C0020A22A1
:1082C000543F4440F51A75190C7518C0020A22541F
:1082D0003F4480F51A75190C7518C0020A22543FE4
:1082E00044C0F51A75190C7518C0020A22740112DF
:1082F0007D997404127D99220000000000000000A6
:10830000000000000000000000000000000000006D
:10831000000000000000000000000000000000005D
:10832000000000000000000000000000000000004D
:10833000000000000000000000000000000000003D
:10834000000000000000000000000000000000002D
:10835000000000000000000000000000000000001D
:10836000000000000000000000000000000000000D
:1083700000000000000000000000000000000000FD
:1083800000000000000000000000000000000000ED
:1083900000000000000000000000000000000000DD
:1083A00000000000000000000000000000000000CD
:1083B00000000000000000000000000000000000BD
:1083C000000000000000000000000000000050520B
:1083D000343032207665722E3132382E332E3120F1
:1083E0004864773A482030362D30372D30352030EC
:1083F000303A30382020004352430000000000197A
:00000001FF
:0300000306028072
